:02000002F0000C
:104000000000042029B10F0051B10F0053B10F007F
:1040100055B10F0057B10F0059B10F00000000005B
:10402000000000000000000000000000C5450F0077
:104030005DB10F00000000005FB10F00954E0F0052
:10404000AD4F0F0063B10F0063B10F0063B10F00FC
:1040500063B10F0063B10F0063B10F0063B10F00D4
:1040600063B10F0063B10F0063B10F0063B10F00C4
:1040700063B10F0063B10F0063B10F0063B10F00B4
:1040800063B10F0005740F0063B10F0063B10F003F
:10409000C1740F0063B10F00894B0F0063B10F00B3
:1040A00063B10F0063B10F0063B10F0063B10F0084
:1040B00063B10F0063B10F000000000000000000BA
:1040C00063B10F0063B10F0063B10F0063B10F0064
:1040D00063B10F0063B10F0063B10F0081860F0061
:1040E00063B10F0063B10F0063B10F000000000067
:1040F0000000000063B10F000000000063B10F007A
:1041000000000000000000000000000000000000AF
:10411000000000000000000000000000000000009F
:10412000000000000000000000000000000000008F
:10413000000000000000000000000000000000007F
:10414000000000000000000000000000000000006F
:10415000000000000000000000000000000000005F
:10416000000000000000000000000000000000004F
:10417000000000000000000000000000000000003F
:10418000000000000000000000000000000000002F
:10419000000000000000000000000000000000001F
:1041A000000000000000000000000000000000000F
:1041B00000000000000000000000000000000000FF
:1041C00000000000000000000000000000000000EF
:1041D00000000000000000000000000000000000DF
:1041E00000000000000000000000000000000000CF
:1041F00000000000000000000000000000000000BF
:1042000010B5054C237833B9044B13B10448AFF310
:1042100000800123237010BDC48600200000000030
:10422000D0B70F0008B5034B1BB103490348AFF3E8
:10423000008008BD00000000C8860020D0B70F0035
:10424000A3F5803A704700BF174B002B08BF134BF4
:104250009D46FFF7F5FF00218B460F461348144A91
:10426000121A00F05FF80E4B002B00D098470D4B50
:10427000002B00D098470020002104000D000D48BD
:10428000002802D00C4800F00FF900F027F82000B9
:10429000290000F097FA00F011F800BF00000800B4
:1042A000000000000000000000000420C486002080
:1042B000A4CE0020A9440F00B5440F0008B500218A
:1042C000044600F08BF8044B1868C36B03B19847A1
:1042D000204600F04FF900BFA8B50F0070B50D4E95
:1042E0000D4D761BB61006D0002455F8043B013462
:1042F0009847A642F9D1094E094D761B07F048F9B7
:10430000B61006D0002455F8043B01349847A64265
:10431000F9D170BDB8860020B8860020C086002084
:10432000B8860020830730B548D0541E002A3FD0FD
:10433000CAB2034601E0013C3AD303F8012B9D07C2
:10434000F9D1032C2DD9CDB245EA05250F2C45EA2C
:10435000054536D9A4F1100222F00F0C03F1200E0E
:10436000E6444FEA121C03F1100242E9045542E907
:10437000025510327245F8D10CF1010214F00C0F05
:1043800003EB021204F00F0C13D0ACF1040323F082
:1043900003030433134442F8045B9342FBD10CF053
:1043A00003042CB1CAB21C4403F8012B9C42FBD17C
:1043B00030BD64461346002CF4D1F9E70346144699
:1043C000BFE71A46A446E0E7024B13B1024800F0EB
:1043D0006BB8704700000000B5440F002DE9F84F9E
:1043E0002F4B2DED028B834618680F4600F078F8AE
:1043F0002C4BD3F80080D8F84861AEB108EE10BA63
:104400004FF001094FF0000A7468651E0CD40134A6
:1044100006EB840487B1D4F80031BB420CD0013DD7
:104420006B1CA4F10404F5D1BDEC028B1C4B186885
:10443000BDE8F84F00F056B873682268013BAB4204
:104440000CBF7560C4F800A0002AE8D0D6F8880137
:10445000D6F804B009FA05F101420BD19047726811
:104460005A4513D1D8F84831B342D8D01E46002E51
:10447000CAD1D9E7D6F88C0101420CD1D4F880100A
:1044800018EE100A904772685A45EBD0D8F8486188
:10449000002EB9D1C8E7D4F880009047DFE700BF0D
:1044A00028840020A8B50F00002301461A461846AC
:1044B00000F01AB838B5084B084D5B1B9C1007D0AC
:1044C000043B1D44013C55F804399847002CF9D1B0
:1044D000BDE8384007F062B8C4860020C0860020DE
:1044E000704700BF704700BF2DE9F047DFF880A09C
:1044F0000646DAF8000098460F469146FFF7F0FFAF
:104500001A4B1B68D3F8484124B365681F2D26DC7D
:104510005EB96B1C0235DAF80000636044F8257060
:10452000FFF7E0FF0020BDE8F08704EB85010123E1
:10453000C1F88890D4F88821AB401A43022EC4F801
:104540008821C1F80881E4D1D4F88C211343C4F840
:104550008C31DEE703F5A674C3F84841D5E7DAF8F5
:104560000000FFF7BFFF4FF0FF30DCE7A8B50F00FA
:1045700028840020FEE700BF38B50C46E8B909687A
:10458000C9B10F4DA9420BD06B1A3B2B11D93C225C
:10459000284606F0F7FD03E0CA5CEA54013BFBD273
:1045A000074800223C2103F091FA0023A8872360EA
:1045B00038BD3D23F2E70E23F9E70123F7E700BFFB
:1045C000807F0020074A6FF002039E4502D1EFF37F
:1045D000098101E0EFF308818869A0F10200007809
:1045E000104700BF79450F0038B50446A8B10D4DFE
:1045F00000223C21284603F069FAAB8F83420ED19A
:104600002A4605F13C0152F8040B44F8040B8A4297
:10461000F9D10133AB87002038BD0E20FCE70B2019
:10462000FAE700BF807F00200B2970B504461546CD
:1046300008462FD92389053304EB43012044431A4C
:10464000DAB2012A26D9814224D8134806F09AFD0D
:104650002388522B06D1AB0711D062884CF66863D1
:104660009A420CD00F2014E034F8022B824204D07E
:10467000AE89964203F1010308D1002009E02189A7
:1046800000230A344FF6FE704FF440559942EBD8A0
:104690000B2070BD0920FCE7E186002008B5002250
:1046A00003F014FA034B1B88834214BF0B20002035
:1046B00008BD00BFE186002038B50C4C21684B1CBA
:1046C000054612D00A484FF4805206F04BFD48B11F
:1046D00015B1206800F0C6FC054920684FF48062DF
:1046E00000F0E0FC4FF0FF33236038BD2C84002045
:1046F000EC8600202DE9F041DFF84480044624F4E4
:104700007F651846D8F8003025F00F05AB420E46FD
:10471000174609D0FFF7D0FF0848C8F800504FF4FB
:104720008052294606F02EFD0448C4F30B043A4695
:1047300031462044BDE8F04106F024BDEC8600205F
:104740002C840020BFF34F8F0549064BCA6802F442
:10475000E0621343CB60BFF34F8F00BFFDE700BFA4
:1047600000ED00E00400FA054BDF704710DF7047F2
:1047700011DF704713DF704718DF704760DF704745
:1047800069DF704761DF70471FB50023CDE9013352
:104790000393684602230093FFF7EEFF05B05DF830
:1047A00004FB08B54FF0E023D3F8F03DDB0700D55C
:1047B00000BEFFF7C7FF0000014B1878704700BF2D
:1047C000ED9600202DE9FF484C4B40F20242C3F821
:1047D000402500F063FA00F0DBFE002000F062FBF1
:1047E00000F056FF48B1052000F05CFB00F062FFCE
:1047F00000F086FF062000F055FB4FF08043DFF805
:104800001081D3F81C55B12D0CBF0123002388F86B
:1048100000304AD0A5F1A8014C424C41384EDFF897
:10482000F49004F0010333704FF08043D3F8007428
:1048300007F00107002C3BD14E2D38D0572D36D034
:10484000304B1B681A68304B9A4200D17FBB6D2DEC
:104850002ED0082000F0B2F9044633789BBB082024
:1048600000F0ACF910B1082000F0A8F900F0010048
:10487000307000F0BFFDDFF8A0B0824630B12CB937
:10488000204B1B681A68214B9A4257D04FF4405373
:104890005A684A450ABF9B684FF4905303F500736A
:1048A0001B685B453AD1012448E00124B6E70124A6
:1048B0004FF0804300226D2DC3F81C2500F0E480EA
:1048C000002CCAD1C5E70120D0E7544636E03C466B
:1048D00034E04FF480030B6071E0022000F0E2FA54
:1048E000A5F14E035842584103F0CEFEAEE000223F
:1048F0001146C1E003F018FFC6E000BF00A0004071
:10490000ED96002030840020D51A5A007E67E54ECF
:10491000EE960020DBE5B1517CB0EE87002CC2D1D1
:10492000BAF1000FD1D0002FD1D0654B654A1B687A
:1049300065481A60654B43F0010398474FF44053B4
:104940005A684A4508BF9B685D4A0CBF03F500736F
:104950004FF4905312681B685B450CBF5C4B0023FF
:1049600013601CB9BAF1000F40F08E803378002B31
:10497000B3D0082000F096FA98F800300BB9FFF792
:1049800003FF01234FF4742088F80030FFF7F2FE94
:10499000504B51491868019001A8FFF7E7FE4F49B5
:1049A00091F816335A09EC231341DA0707D54C4B1B
:1049B0009A68002A8DD01A6842F480021A600C228C
:1049C000484B029300210DEB0200FFF7ABFC40F2D5
:1049D0000113029A039303A94020FFF7D1FE0C2292
:1049E00000210DEB0200FFF79DFC9DF80C30029AB0
:1049F00043F0010303A9A0208DF80C30FFF7C0FE9F
:104A00000C2200210DEB0200FFF78CFC0124F723A0
:104A1000029AADF80E3003A923208DF80C40FFF761
:104A2000AFFE0C2200210DEB0200FFF77BFC0623FA
:104A3000029A8DF80C4003A920208DF80E40ADF8A5
:104A40001030FFF79DFE02A8FFF798FE4FF4405389
:104A500030785A684A450ABF9B684FF4905303F573
:104A600000731B685B4504D0572D02D04E2D7FF498
:104A70003EAF012240F6B83100F0A2FD3378002BA2
:104A80003FF438AFFFF774FE00F086F900F0B2FC97
:104A9000A0B100F0FDFD88B94FF440535B684B4571
:104AA00006D198F800300BB9FFF76EFEFFF760FEF5
:104AB000034B1B6800221A6000F0BEFDFFF742FEA8
:104AC00030840020D51A5A000048E801B0B50F0024
:104AD0007E67E54EACB50F00A3470F0000E100E094
:104AE000409D00200080002010B5FEB04FF4FA7306
:104AF000ADF802300DF10201002301A8ADF8043039
:104B0000FFF740FE044640B9BDF80430102B07D033
:104B1000112B0CD001A801F085F820467EB010BD05
:104B2000054B01221A70072000F0BCF9F2E7024B96
:104B300018700820F8E700BFEC96002013B500239A
:104B400001A80193FFF710FE044660B9019802F036
:104B50000FFB019B0A2B09D0092B09D00B2B02D18B
:104B6000012004F0DFFB204602B010BD2046F8E72C
:104B70000220F6E708B5FFF7B7FF0528FBD1FFF7DE
:104B8000DDFF0528F7D108BD0021024A084602F0E2
:104B9000BFBE00BF754B0F001F2884BF00F01F0071
:104BA000044B054A98BF4FF0A04300F5E07043F86E
:104BB00020207047000300500C0003001F288ABF0C
:104BC000064B4FF0A04300F01F00D3F8103523FA36
:104BD00000F0C04300F00100704700BF0003005028
:104BE00000234FF0FF328360C0F80035C0F8602525
:104BF000C0F86425C0F86825C0F86C2540F2FF3283
:104C0000C0F80435C0F80825C0F80C35C0F81035D8
:104C1000C0F81435C0F82035C0F8243570470000BE
:104C20001B4B00221F2930B5C3F800258BBF01F0B4
:104C30001F030B46174A4FF0A04203F5E07403250B
:104C400042F82450012404FA03F3C2F80C3500F5AD
:104C5000AC700F4B002243F82010FF21C3F804254D
:104C60000220C3F808150421C3F80C15C3F8100579
:104C70000948C3F81425C3F82005C3F82415C3F860
:104C80002825C3F82C25C3F80045C3F8102130BDF2
:104C900000C0014000030050E498002038B54FF0F8
:104CA000804301240025DC600820C3F818559C606F
:104CB000FFF772FF0820FFF76FFF2E4B4FF4C8502D
:104CC0002343984723212846FFF7AAFF24212046A3
:104CD000FFF7A6FF4FF01023D3F8043303F00703C8
:104CE000052B25D0244AC2F80445D2F80034002B05
:104CF000FBD04FF01021D1F8043323F0070343F029
:104D00000503C1F804330023C2F804351A4AD2F867
:104D10000034002BFBD0BFF34F8F1849184BCA68E3
:104D200002F4E0621343CB60BFF34F8F00BFFDE797
:104D3000144A1E21082002F0C7FD08B102F07EFED1
:104D400002F028FD0D49104BE02081F823001B687C
:104D50004FF47A72B3FBF2F3013BB3F1807F08D2D8
:104D60004FF0E0225361002381F823009361072371
:104D7000136138BDC0B50F0000E0014000ED00E058
:104D80000400FA05F0960020348400200148FFF763
:104D900027BF00BF00C001404FF0E023002110B545
:104DA0001961FFF7F3FF144B144C4FF40032C3F8B2
:104DB000802003F1C04303F53C534FF48032C3F825
:104DC0004823C3F8082301225A609A604FF08043B9
:104DD0000220DA600B461F2B1A46C6BF03F01F02E3
:104DE00021464FF0A04102F5E0720133302B41F82B
:104DF0002200F0D110BD00BF00E100E00003005030
:104E0000074B23F81010074B002282B0C3F8102183
:104E1000D3F810210192019A01229A6002B07047E2
:104E2000E498002000C0014010B5174B1C68174BD8
:104E30001B68B4FBF3F103FB1141B1EB530F88BFC7
:104E4000591A5A084F235943B1FBF2F1C1F1FF013E
:104E500089B20020FFF7D4FF0D4B1B68B4FBF3F1C0
:104E600003FB1144B4EB530F4FEA530188BF1C1BE3
:104E70008F235C43B4FBF1F1C1F1FF01BDE81040A9
:104E800089B20120FFF7BCBFE0980020EC98002019
:104E9000F4980020024A136801331360FFF7C4BF7F
:104EA000E09800201B490A68082823D8DFE800F0B2
:104EB00013051322221A1E242A00174B40F6B8307D
:104EC00018604FF47F4303F0103323F080539A426D
:104ED00018BF0B607047104B4FF4967018604FF47A
:104EE0007F03F0E70C4B64221A6070470A4B40F6D0
:104EF000B83018601346E6E7084B40F6B830186043
:104F0000FF23E0E7054B4FF4967018604FF0FF1356
:104F1000D9E700BFF0980020EC980020F49800201A
:104F200000F1804382B01A68002A14BF01200020DB
:104F300004D000221A601B680193019B02B07047E5
:104F40000F4A1378D3B903784FF08041C3F340037D
:104F5000C1F88035037803F00103C1F87835094BB7
:104F60001968C90706D4E02183F800130121C3F8AA
:104F7000801119600123044813707047034870477B
:104F80000499002000E100E00000AD0B0C00AD0B27
:104F9000014B02681A607047009900204FF080436F
:104FA0004FF46072C3F804237047000010B54FF04F
:104FB0008043D3F80443620707D54FF48470FFF7AA
:104FC000AFFF10B11E4B1B689847A30608D54FF4DE
:104FD0008A70FFF7A5FF18B11A4B00201B6898478D
:104FE000600608D54FF48C70FFF79AFF18B1154B87
:104FF00001201B689847210608D54FF48E70FFF7F3
:105000008FFF18B1104B00201B689847E20508D5A8
:105010004FF49070FFF784FF18B10B4B01201B6811
:105020009847A3050AD54FF49270FFF779FF28B18E
:10503000054BBDE810401B680220184710BD00BF9B
:10504000F8980020FC98002000990020044AD2F82B
:105050000034DB07FBD50160BFF35F8F704700BFF3
:1050600000E001404FF080531A69B0FBF2F302FBFD
:10507000130373B9084B0222C3F80425C3F80805CB
:10508000D3F80024D207FBD500220448C3F8042536
:1050900070470348704700BF00E001400000AD0BBF
:1050A0000A00AD0BF8B50B4B1546012206460F461C
:1050B000C3F804250024A54204D1064B0022C3F8FE
:1050C0000425F8BD57F8241006EB8400FFF7BEFF57
:1050D0000134F0E700E00140BFF34F8F0549064B74
:1050E000CA6802F4E0621343CB60BFF34F8F00BF86
:1050F000FDE700BF00ED00E00400FA054FF080532B
:10510000D3F83021082A06D1D3F83431032B02D842
:10511000024AD05C70470020704700BFC6B50F0040
:1051200008B54FF08053D3F83021082A4ED14FF004
:1051300080420021C2F80C11C2F81011C2F83815D3
:1051400002F54042D3F80414C2F82015D3F808142D
:10515000C2F82415D3F80C14C2F82815D3F810148B
:10516000C2F82C15D3F81414C2F83015D3F818145B
:10517000C2F83415D3F81C14C2F84015D3F8201423
:10518000C2F84415D3F82414C2F84815D3F82814EB
:10519000C2F84C15D3F82C14C2F85015D3F83014BB
:1051A000C2F85415D3F83414C2F86015D3F8381483
:1051B000C2F86415D3F83C14C2F86815D3F840144B
:1051C000C2F86C15D3F84434C2F87035FFF796FF77
:1051D00018B1494B494AC3F88C26FFF78FFF18B125
:1051E000474BFB22C3F81825FFF788FF70B14FF03B
:1051F00080414FF08053D1F8E42ED3F8583222F09A
:105200000F0203F00F031343C1F8E43EFFF776FFEC
:1052100020B13C4B4FF40072C3F840264FF080534E
:10522000D3F83031082B09D14FF08043D3F8002454
:10523000D10744BF6FF00102C3F80024324AD2F80C
:10524000883043F47003C2F88830BFF34F8FBFF348
:105250006F8F4FF01023D3F80C22D2071DD52B4BA4
:105260000122C3F80425D3F80024002AFBD04FF014
:105270001022D2F80C3223F00103C2F80C32234B77
:10528000D3F80024002AFBD00022C3F80425D3F869
:105290000024002AFBD0FFF71FFFD3F80022002ACA
:1052A00003DBD3F80432002B22DA184B0122C3F8B7
:1052B0000425D3F80024002AFBD04FF0102212213D
:1052C000C2F80012D3F80024002AFBD04FF01023BC
:1052D0001222C3F804220D4BD3F80024002AFBD07D
:1052E0000022C3F80425D3F80024002AFBD0D2E71B
:1052F000074B084A1A6008BD00500040488103006F
:1053000000F000400090024000ED00E000E00140AD
:10531000348400200090D00313DF704718DF7047FB
:10532000064B1878012803D1012904BF0221197006
:1053300012B1104602F082BB704700BF35990020C1
:1053400008B5FFF739FA88B111481C2101F09CFF1C
:1053500008B102F073FB0F490D4800231C2201F035
:1053600083FF98B1BDE8084002F068BB4FF47F208E
:10537000FFF778FE072207494FF47F20FFF792FEE0
:10538000054B1A78012A04BF02221A7008BD00BF1B
:105390002C990020389900203599002070B5124CC6
:1053A000124D134ED4F800347BB1C4F80056C4F843
:1053B0000456C4F80856C4F80C56C4F81056C4F87D
:1053C0001456C4F81856C4F81C5602F009FB05F030
:1053D000A8FE20B104F060FD002005F049F9337803
:1053E000023B022BDED870BD000001403546526EF4
:1053F0003599002013B54FF44053124A5968914231
:105400000CBF9C684FF4805401A800F0A7F92368F2
:10541000013302D16368013311D0019B1A88012A3C
:105420000DD1588820B199680022204602F04EFB29
:10543000019B5B881B1A5842584102B010BD0020E6
:10544000FBE700BFDBE5B15184B02DE9F34108ACC7
:1054500084E80F009DF82040BDF8228001A80F4687
:1054600016461D4600F07AF954B9384B0122FF2147
:10547000A3F802809D601A809980354B1A7012E063
:10548000012C17D1314BBA192A449A60A5221A80EF
:10549000FF229A800C9AA3F80280C3E903765D612B
:1054A0009A612B4B1C70FFF74BFF02B0BDE8F04137
:1054B00004B07047032C0FD1019A244B1188198036
:1054C000518892689A60C3E90376AA2259809A802B
:1054D0005D611F4B0122D1E7022C15D1019A1B4BB4
:1054E0001188A5290AD100229A60FF221A60FF22A2
:1054F0009A800022C3E903225A61EAE719805188A1
:10550000926859809A60F2E7052C0ED1FFF754F9A2
:1055100040B100F09BFD08B102F090FA0C4B032261
:105520001A70C2E700F010FAF5E7042C08D1074B17
:1055300000229A60FF221A60019A92889A80B2E74C
:10554000062CB2D1024B0422EAE700BF38990020B2
:105550003599002000B50C4B1B7889B063B90B4B13
:105560001B786BB905238DF80C30079B009303ABB8
:105570000FCBFFF769FF03E004F08AFA0028EED0B2
:1055800009B05DF804FB00BF349900202899002081
:105590001FB50023CDE90233074B019301F034FE20
:1055A00030B906494FF47F2301A84B6001F04AFE51
:1055B00005B05DF804FB00BF21530F002C990020BB
:1055C00070B505460E460AB180F00102154B02F097
:1055D00001021A7000F0B4FF044628B935B100F09A
:1055E0008BFC0446FFF7DAFE204670BDBEB10E4BC1
:1055F0000E4A0F481D70294602F0FCF84FF4004493
:105600004FF4FA7029464FF47A720023E6FB040146
:1056100005F03CFE2A460146064802F0FDF800F07F
:105620006FF9DEE7349900202899002055550F00C6
:10563000CCB50F00089900201FB5134B4FF0FF3277
:10564000C3F88020C3F880214FF440530F4A5968B3
:1056500091420DD19C682046FFF75EFE10B14FF0DD
:1056600000531C60204604B0BDE8104000F09AB81A
:105670000023CDE902334FF4805406236846CDE978
:105680000034FFF74BFEE9E700E100E0DBE5B15154
:1056900007B501A800F062F8019B1A88A52A07D077
:1056A0009888A0F1AA035842584103B05DF804FB62
:1056B0000120FAE710B501F061F9A8B10E4B0F48CF
:1056C00043F00103984701F0C3F808B102F0B6F9BE
:1056D00001F054F908B102F0B1F901F005F90446FE
:1056E00038B102F0ABF904E001F022F904460028D9
:1056F000E4D1204610BD00BFD0B50F0000A8610066
:1057000000B589B003AB142200211846FEF70AFE4B
:1057100002228DF80C20002200920FC8FFF794FEA1
:10572000FFF73CFE002009B05DF804FB13B504460A
:1057300001A800F013F8019B1A8822805A88628021
:105740009A68A2609A88A280DA68E2601A69226187
:105750005A6962619B69A36102B010BD014B03608D
:10576000704700BF00F00F00F0B50346186880F3E3
:1057700008885868FF2464B2EFF30585002D01D135
:10578000A64600472546064621273FBAF0B4002426
:10579000002500260027F0B4F92040B2004700BFE2
:1057A000F0BD00BFFFF7E0BF73B500230DF10201AC
:1057B00001A8ADF80230019302F0C8FDF8B9019CD0
:1057C00025785DB3174B93F83020032A28D00C2698
:1057D00006FB00F29958E9B998189D5093F83020CB
:1057E0000132D2B283F83020BDF802300E4A9B0855
:1057F000013B043443608460084602F089F8019B51
:1058000033B128B1184602F0BDFD08B102F016F917
:1058100002B070BD01300428DAD1F0E70720EEE7CE
:105820000420ECE75499002071580F00084609B194
:1058300002F004B97047000010B50C220B4B504326
:1058400019181A5882B193F830208C68013AD2B2F4
:1058500083F8302000221A50C1E90122201F02F0F3
:1058600091FD08B102F0EAF8002010BD5499002023
:10587000214B70B50122214E1A7096F8303003B9D1
:1058800070BD1E4C0025236883B1013B042B07D853
:10589000DFE803F01C0612032800204600F0E2FEB9
:1058A000E8B2FFF7C9FF08B102F0C8F80135042DCE
:1058B00004F10C04E7D1E0E7A3686360204600F040
:1058C00077FE0028ECD002F0B9F8E9E7204600F0B6
:1058D00057FF00F033FF08B102F0B0F80520FFF7E2
:1058E000E1FADDE700F078FF00F096FFBDE87040D8
:1058F0000620FFF7D7BA00BF28990020549900204E
:1059000008B50E4B002283F8302004210139C3E989
:1059100001221A6003F10C03F8D1094800F042FE9D
:1059200002F0ACFC08B102F089F8064802F092FCE3
:1059300008B102F083F8002008BD00BF5499002090
:105940002D580F00A9570F0008B50020FFF774FF6E
:105950000120FFF771FF0220FFF76EFF0320FFF722
:105960006BFFBDE8084002F0D1BC006870476CDFF7
:1059700070476DDF70476EDF70476FDF704772DF13
:10598000704773DF704774DF704776DF704777DFEB
:1059900070477ADF70477CDF70477FDF704786DFB4
:1059A00070478FDF704790DF7047AFDF7047B0DF21
:1059B0007047B1DF7047B2DF7047B5DF704764DF13
:1059C000704766DF70470C2813D8DFE800F0141228
:1059D0001212121209120712120D0B000220704748
:1059E0000320704704207047042914BF06200520B7
:1059F0007047062070470120704702F01FB810B5AD
:105A0000044608460321FFF7DEFF0246204601F068
:105A100079F918B1BDE8104002F010B810BD0000CF
:105A20000346032B10B50846144620D0042B23D17F
:105A300069B1124B18884FF6FF7398421CD013219E
:105A4000FFF7A3FFC0B1BDE8104001F0F7BF10465B
:105A500002F098F808B101F0F1FF094B1B689C4275
:105A60000AD101220321074801F04CF9EAE701219C
:105A7000FFF7A9FF0246F6E710BD00BF3A840020F9
:105A8000489A0020F8990020F8B50A4DAB889E1876
:105A90001D2E14460DDC2F68FE1802F1010C07F8CC
:105AA00003C07070B01C05F06DFBAB8802331A198F
:105AB000AA80F8BDA8990020F0B54E4E317895B077
:105AC000002940F092804C4C019110222046FEF7B4
:105AD00029FC4A4B0199236018220EA8FEF722FCEC
:105AE00001238DF8383028231093454B1B78002B69
:105AF0007DD0444B04AC03F1100518685968224668
:105B000003C20833AB421446F7D13F4C10220DEBD1
:105B10000201E01D05F026FB002868D03B4801216A
:105B20000460FFF728FF08B101F088FF384B08AA8E
:105B300003F1100C174618685968154603C5083359
:105B400063452A46F7D120680C903248A288A37991
:105B5000ADF834200760012200218DF83630FFF7C0
:105B60000CFF08B101F06AFF03238DF84C300423C9
:105B70008DF80E3041F23053ADF81030264B08AAA4
:105B80009B798DF812300DF10F0104A8FFF717FF74
:105B9000012210460DF10E01FFF776FF1F4805F0B8
:105BA00028FB1E49C2B20920FFF76EFF102208A988
:105BB0000620FFF769FF104919480EAAFFF7DFFE1C
:105BC00008B101F03BFF164C042221780120FFF7B9
:105BD000DEFE08B101F032FF20780121FFF7D1FE8F
:105BE00008B101F02BFF0123337015B0F0BD06237F
:105BF000BEE700BF2C9A0020A899002088990020B9
:105C0000F49900200CB60F00B8990020449A0020A7
:105C1000BF990020289A0020F8990020D6B50F00DF
:105C200038840020F0B504460146B1B0A84801F020
:105C30009DF82388262B3BD80F2B04D8012B00F08E
:105C4000CC8031B0F0BD103B162BFAD801A252F82F
:105C500023F000BFDD5C0F00EB5C0F00435C0F0026
:105C60001D5D0F00175E0F00435C0F00435C0F00CB
:105C7000435C0F00435C0F00435C0F00335E0F007A
:105C8000435C0F00435C0F00435C0F00435C0F005C
:105C9000435C0F00435C0F00A95E0F00435C0F00E4
:105CA0009B5E0F00435C0F00435C0F009D5D0F0087
:105CB000513B9AB2052AC4D8052BC2D801A252F88A
:105CC00023F000BFE75D0F00335E0F00435C0F0061
:105CD000435C0F00BF5E0F00835D0F007D4BA28809
:105CE0001A807D4B00221A70ABE78023794CADF807
:105CF00024307A4B208832221A6010A9012309AA85
:105D0000FFF759FE08B101F099FE754B1B780BB9EE
:105D1000FFF7D2FE4FF6FF73238092E7714B03AC7F
:105D20009A79186899888DF822200790DA1DADF8C5
:105D300020101733264610685168254603C50832DF
:105D40009A422C46F7D1684B09AA03F11807154669
:105D500018685968144603C40833BB422246F7D179
:105D6000186820605B48614A008810AB8521CDE946
:105D70001456FFF712FE00283FF463AF01F05EFEF9
:105D80005FE7A379002B7FF45CAF524B1321188897
:105D9000FFF7FBFD00283FF454AF79E0237A012B95
:105DA0007FF44FAF4C4B00221A704C4B19680139ED
:105DB000196069B910AB14221846FEF7B3FA052230
:105DC0008DF84020149A00920FC8FFF73DFB38E78A
:105DD00031B0BDE8F040FFF76FBE3E4B00211888A0
:105DE000FFF7EFFDD6E7A379002B3FF42AAFA27BA4
:105DF000043A022A3FF625AF022B18BF01238DF883
:105E000040304FF4C173ADF84430324B10A91888BC
:105E1000FFF7CDFDAFE7334A258A508D02F1180117
:105E20000023854218BF19460732A088FFF7B7FD47
:105E3000B0E7284B1C884FF6FF75AC4227D02C4B9F
:105E40001B78F3B12B49012308222046FFF7B1FD4F
:105E5000F0B90246014602232046FFF7AAFDB8B971
:105E60002A460C212046FFF7A0FDA0F54053023B37
:105E7000012B7FF6E6AE08283FF4E3AE112889D166
:105E8000DFE61A4619462046FFF793FD82E7082011
:105E900031B0BDE8F04001F0D1BD0E4B00221888B2
:105EA0001146FFF780FD75E700238DF840308DF82F
:105EB0004130084B10A91888FFF773FDC1E6E1884F
:105EC000044BF729188828BFF721FFF776FD61E713
:105ED000F89900203A8400202C9A00203C8400206D
:105EE0003F9A0020B8990020D09900203A9A0020CB
:105EF000F4990020EC99002030B5474A4748002328
:105F00001370474A95B0137000F04CFB01F0FAFD96
:105F10000446002869D14348FEF766FB002867D194
:105F2000414B01221A70112340488DF8043005F0CE
:105F300060F93E4982B201A8FFF72DFD08B101F0DA
:105F40007DFD0822002104A8FEF7ECF90823ADF836
:105F500010301823ADF812300023ADF8143004A827
:105F60004FF4C873ADF81630FFF713FD08B101F018
:105F700065FD00210C2201A8FEF7D4F90823ADF835
:105F800004302B4B02932B482B4B039301A900F0B9
:105F900033FD08B101F052FD284D4022002104A834
:105FA000FEF7C0F9284605F024F90595244DADF813
:105FB0001000284605F01DF90795224DADF8180090
:105FC000284605F016F91123ADF8300004A8ADF805
:105FD0004C300D9500F0DEFF1B4B30221A7007226B
:105FE0005A7010229A70FFF767FD204615B030BD39
:105FF00004A8FFF7BEFC08B101F020FD9DF81130A8
:1060000004A801338DF81130FFF7B1FC00288AD0C5
:1060100001F014FD87E700BF3F9A0020215A0F00CE
:10602000399A0020B8990020F4990020D6B50F00C5
:106030009D600F00F8990020FB590F00DDB50F009F
:10604000E9B50F00FAB50F003A9A002010B50F4BD2
:1060500001221A700E4B18884FF6FF73984207D032
:106060001321FFF792FC08B101F0E8FC002010BDFD
:10607000084C2378002BF9D0074B1878FFF783FCE6
:1060800008B101F0DBFC00232370EFE73F9A00200A
:106090003A8400202C9A002038840020F0B50B7838
:1060A00089B005460C46092B35D8DFE813F02D00E2
:1060B000360041000A0019002600070110014400C3
:1060C000150100F089FB0421FFF77DFC02462846FC
:1060D00000F018FEF8B109B0BDE8F04001F0AEBC28
:1060E000FFF7B4FF08B101F0A9FC00F095FB90B1F7
:1060F00009B0BDE8F04000F09DBBFFF7A7FF002806
:10610000F6D001F09BFCF3E7764B01221A704B6846
:106110001A78754B1A7009B0F0BD724B02261E70CA
:106120004B681B78012BF6D100F008FB3146CBE71A
:106130006C4B0322EEE70520FEF7B4FE694B1E7898
:10614000022E37D0032E59D0012EE4D104AB1022F9
:1061500018460021FEF7E6F8634A237A12788DF894
:106160001020002203920C2B4FF00302CDE90120F6
:1061700008D03146284600F0C5FD0028CBD001F0FC
:106180005DFCC8E763681846FFF7EFFB0590181D34
:10619000FFF7EBFB069003F10800FFF7E6FB079023
:1061A00001A800F005FA0028B5D03146FFF70BFC36
:1061B0000246DFE7237A13F0030011D0C0F1040296
:1061C0001A44D2B219464FF0000C0E4601316768EE
:1061D000C9B2914207F806C0F7D11B1A04332372E3
:1061E0000123049363680693237A04A89B0805930C
:1061F00000F0C6FA00288ED00221D7E7207A830764
:1062000002D03246314662E7384E0190314601F005
:106210008FFC014618B12846FFF7F1FB7BE7616868
:10622000019A306804F0AEFF019801F0E7FC0146E6
:106230000028F0D101A9304601F0F0FC0146002809
:10624000E9D104230493019B9B08059304A83368B8
:10625000069300F007FA074640B9254A237A1168E9
:106260000B441360234B32681A6054E709281BD192
:106270001F4B217A1A68114419601F4B1B78002BA1
:106280003FF449AF1D4C2388013B9BB22380002B78
:106290007FF441AF284600F0FBFC08B101F0CEFBD3
:1062A000174B1B88238036E7306801F06BFC0146F2
:1062B00010B12846FFF7A3FB3946ACE70E4B01228D
:1062C0001A700F4A8B8813800C4A138023E70A4AFE
:1062D000002313700A4AF8E7054B196800F09CFC8C
:1062E000F8E600BF399A0020409A00204C9A00201E
:1062F000309A0020489A0020389A0020369A0020D0
:10630000349A002018DF7047012973B514460D46F2
:106310001A4608D0032912D014B3204602B0BDE8B3
:10632000704001F08BBB0F4B1B78052BF4D10E4B4B
:106330001B68002BF0D0214604209847ECE7094E5B
:106340003378022BE8D1094B01925B689847064BE2
:1063500035701B68002BDFD0019A21462846ECE7F8
:1063600002B070BD589A0020509A00205C9A00201C
:1063700030B589B003AC142200212046FDF7D2FFCE
:10638000094B1B88ADF80E30084BDB6806930025DF
:10639000079B8DF80C50009394E80F00FFF754F81A
:1063A000284609B030BD00BF689A0020B49A00208A
:1063B00000B589B003238DF80C300A4B1B88ADF86B
:1063C0000E30094B5A6804929A68DB680693079B63
:1063D0000093059203AB0FCBFFF736F8002009B00E
:1063E0005DF804FB689A0020B49A002000B589B0DB
:1063F00001238DF80C300F4B0F4A1B88ADF80E307F
:106400004FF440535968914208BF9A680B4B596842
:10641000049118BF4FF480529968DB680693059188
:10642000009203AB0FCBFFF70FF8002009B05DF827
:1064300004FB00BF689A0020DBE5B151B49A00204C
:1064400000B589B003AB142200211846FDF76AFF9E
:1064500004228DF80C20002200920FC8FEF7F4FFF2
:1064600009B05DF804FB0000194BF7B5194C1C602E
:10647000194B02221A70FEF79FF9184B48B11968A0
:10648000204600F001FF00B303B0BDE8F04001F08A
:10649000D5BA1D68124F013D2D0B013504464FF44E
:1064A00040567368BB420CBFB0684FF4805000EB9D
:1064B00004300134FEF7D6FDA542F2D8002305488A
:1064C00000931A460321FFF71FFF03B0F0BD00BF82
:1064D000CC9A0020C49A0020589A00206C9A002080
:1064E000DBE5B15170B50C4686B00321CDE9021051
:1064F0000546960802A8019304940596FFF702FF4B
:10650000E0B1B4F5805F019B11D8012302A8CDE969
:106510000235CDE90446FFF7F5FE78B9032302A85A
:10652000CDE90235CDE90446FFF7ECFE06E01A4658
:10653000E11AE81AFFF7D6FF0028E6D006B070BDD2
:106540001FB5114B0193114B114900241C70114BC5
:1065500001A81C80CDE9024400F074FE0E4B10B17E
:106560001C7004B010BD4FF440520C4954688C426A
:1065700007490CBF92684FF480524A60084A0021D4
:10658000116001221A70ECE709630F00B09A002035
:10659000C49A0020689A0020589A0020DBE5B15187
:1065A000549A0020014B1860704700BF509A002099
:1065B00038B54368214C0FCB84E80F002278500790
:1065C00001D5910733D16068830730D1A3689D0757
:1065D0002DD1E16811F0030429D118440844184969
:1065E000B3F5204F086024D84FF4405315495D6837
:1065F0008D420ABF9B684FF46923C3F56A23984212
:1066000017D8114B1149196011495960D10709D5A3
:10661000104A9A60104B1B78012B0CD1FFF724FF16
:10662000204638BD92074CBF0C4A0D4AF1E70624BC
:10663000F6E70C24F4E70824F2E700BFB49A002040
:106640006C9A0020DBE5B1515C9A002069640F0070
:1066500041640F00ED630F00589A0020B1630F00F2
:1066600071630F002DE9F04385B0002853D0816895
:1066700011F0030451D12C4B1B78052B4FD12B4E1D
:1066800042683368DFF8AC9003EB82039500D9F8D9
:106690000020934207D94FF0FF3333600C2420468B
:1066A00005B0BDE8F0830391FEF786F8DFF8888037
:1066B000039940B13368D8F800002A4600F0D4FDB1
:1066C000D8B10446EBE74FF44053194A586837688D
:1066D000904208BF9868039118BF4FF48050002380
:1066E0002A463844FEF706F80399D8F800000095CA
:1066F0000B4600220121FFF707FE33681D44D9F83D
:10670000003035609D420CD1FEF756F80028C6D106
:10671000FDF7D2FFC3E70E24C1E71024BFE708242A
:10672000BDE70924BBE700BF589A0020549A002017
:10673000DBE5B1516C9A0020CC9A002070B50B4B70
:106740001D6885B90A4E3378042B0CD1094C0A4BCD
:1067500021781A780948FDF767FF10B905233370CF
:1067600070BD2570FCE70820FAE700BF549A0020AE
:10677000589A0020B09A0020B49A0020709A002005
:10678000F8B5114B1A78032A03D0042A03D0082441
:1067900016E004221A700D4B1C68002CF7D10C4D2A
:1067A00043682F789E0007EB8303402B0AD881684B
:1067B00008483246384404F0E5FC2B7833442B700B
:1067C0002046F8BD0924FBE7589A0020549A00207F
:1067D000B09A0020709A002010B50B4C2378052B3E
:1067E00010D10A4B0A4A1B68116899420AD1062344
:1067F0002370084B1B685868FDF750FF08B9072342
:10680000237010BD0820FCE7589A00206C9A0020E5
:10681000549A0020CC9A0020044B1B78072B02D1FD
:10682000034B9B6818470820704700BF589A002008
:106830005C9A002000B589B006238DF80C30079BC8
:10684000009303AB0FCBFEF7FFFD09B05DF804FB2F
:10685000F0B58DB005A8FEF769FF089C002C3ED06E
:106860000B9E04F58053B3422DD91E4BA6F58055DF
:1068700003EA55054FF440539B689C420BD86900CE
:106880002B46A4EB450201F5805106EB4500FFF7CE
:1068900029FE0DB0F0BD05F58053012701A8CDE913
:1068A0000173CDE90337FFF72DFD0028F1D14FF437
:1068B000805301A8CDE9023301970497FFF722FD29
:1068C0000028E6D1DBE70123CDE90136A4084FF427
:1068D000805301A803930494FFF714FDD9E72046E1
:1068E000D7E700BF00F0FFFF00B58DB005A8FEF7A9
:1068F0001DFF099880B1089B8BB94FF440530B4A98
:10690000596891420ED19B6880080022039001A82B
:10691000CDE90123FFF7F6FC0DB05DF804FB0B9AFF
:106920001344F1E74FF48053EEE700BFDBE5B151CC
:1069300000B58DB005A8FEF7F9FE099898B1089B3F
:10694000A3B94FF440530C4A5968914211D19B6846
:106950000393800803214FF47422049001A8CDE929
:106960000112FFF7CFFC0DB05DF804FB0B9A134446
:10697000EEE74FF48053EBE7DBE5B15110B58CB097
:1069800005A8FEF7D3FE0898B8B10B9C00F580531C
:10699000A34214D94FF440539B6898421BD80F4B25
:1069A000A4F5805203EA52035900A0EB430201F51B
:1069B000805104EB4300FFF795FD0CB010BD80083B
:1069C00003224FF48053049001A8CDE901230394DE
:1069D000FFF798FCF1E70E20EFE700BF00F0FFFFA4
:1069E000A8DF7047AADF7047ADDF7047AEDF7047A2
:1069F000B0DF704762DF70472DE9F0470E4694B074
:106A00000546002800F00181002900F0FE804B6857
:106A1000002B00F0FA804FF6FF7303800023ADF8DF
:106A20000A307B4B04AA03F1100C1746186859680A
:106A3000144603C4083363452246F7D141F230536C
:106A40000DF10A013846ADF80830FFF7D3FF0446D0
:106A5000002840F0D6802A1D02A90120FFF7C0FFC0
:106A60000446002840F0CD809DF80A30AB71014605
:106A70001C220DA8FDF756FC9DF834300E9443F00F
:106A800004038DF8343001AFAB798DF80E30214618
:106A900041F2325303223846CDE91044CDE9124485
:106AA000ADF80C30FDF73EFC9DF806308DF8044043
:106AB00023F01F0343F00303214614224FF0110A71
:106AC00008A88DF806308DF805A00DF10C08FDF72B
:106AD00029FC4FF01409A8880A9405F1080308AAB4
:106AE0000DA90C94CDE90887ADF82C90FFF77AFF3B
:106AF0000446002840F0858001461C220DA8FDF7C1
:106B000011FC9DF834300E9423F0180343F0180361
:106B10008DF83430AB798DF80E30214641F2315387
:106B200003223846CDE91044CDE91244ADF80C30CB
:106B3000FDF7F8FB9DF806308DF8044023F01F03A5
:106B400043F0130321464A4608A88DF806308DF815
:106B500005A0FDF7E7FB1723ADF82C30A8880A94B1
:106B600005F1100308AA0DA90C94CDE90887FFF7D9
:106B700039FF0446002844D101461C220DA8FDF728
:106B8000D1FB9DF834300E9443F002038DF834307D
:106B9000AB798DF80E30214641F23453032238464A
:106BA000CDE91044CDE91244ADF80C30FDF7BAFB45
:106BB0009DF806308DF8054023F01F0343F00303D2
:106BC00021464A4608A88DF806308DF804A0FDF746
:106BD000A9FB02230A93ADF82C30A8880C9605F186
:106BE000200308AA0DA9CDE90887FFF7FBFE04469C
:106BF00038B97368AB62B36803B1EB62054B01222D
:106C00001A70204614B0BDE8F0870E24F9E700BFE3
:106C10001CB60F00D09A002070B5054686B070B340
:106C200002884FF6FF739A422BD0174B1B7843B361
:106C3000164C1022080AE170207121FA02F0090EA8
:106C4000072301266071A17102A800216370ADF8CD
:106C500006302270A670FDF765FB2B8AADF8083070
:106C60000023ADF80C3028888DF80A600DF106037A
:106C700002A9CDE90434FFF7B9FE06B070BD0E20BD
:106C8000FBE70820F9E700BFD09A0020D19A002046
:106C900030B5044687B060B302884FF6FF739A425E
:106CA00029D0164B1B7833B3154D11232B700B0ACB
:106CB0006970AB700B0C090EEB7029710523002174
:106CC000102202A8ADF80630FDF72CFB238AADF8A0
:106CD000083001238DF80A300023ADF80C302088ED
:106CE0000DF1060302A9CDE90435FFF77FFE07B0D9
:106CF00030BD0E20FBE70820F9E700BFD09A002046
:106D0000D19A002030B5044687B038B300884FF6DA
:106D1000FF73984224D0134B1B780BB3124D1023F2
:106D200069700321ADF80610AA7000211A4602A866
:106D30002B70FDF7F7FA238AADF8083001238DF8A0
:106D40000A300023ADF80C3020880DF1060302A9AB
:106D5000CDE90435FFF74AFE07B030BD0E20FBE752
:106D60000820F9E7D09A0020D19A002070B50D468E
:106D700088B0044650B149B1826A3AB10B88502BB1
:106D800049D005D8102B43D0112B54D008B070BD7A
:106D9000512BFBD18E79022EF8D10A89038A9A42AF
:106DA000F4D18B7B043B022BF0D99DF816308DF883
:106DB000106043F001038DF816300B8AADF81830DF
:106DC0004B8AADF81A30082201F1140301A8002102
:106DD0000793FDF7A7FAA18A2088019601AACDF8AA
:106DE00008D0FFF701FE48B3E36A03B1984740F2C9
:106DF000FD132088ADF8143004A9FFF7F9FD002831
:106E0000C4D0E36A002BC1D008B0BDE87040184779
:106E10008B882380BAE7C98803899942B6D10823B1
:106E20008DF81030123535F8023C8DF81830059584
:106E300004A99047AAE74FF6FF73EAE7BDF80030D0
:106E40002088DB07D3D5002604A9ADF81460FFF72E
:106E5000CFFD0028D5D1297D4B1E072B3ED8DFE87A
:106E600003F004192226282A3B2C6B8A8DF8046033
:106E7000012B05D8062201212046FFF743FFBEE77C
:106E8000012315358DF80C300295A36A01A920461F
:106E900098477BE76A8A01239A428DF80430F0D83C
:106EA00006220221E8E702238DF80430EDE70323F0
:106EB000FAE70423F8E70523F6E76B8A022B02D8EA
:106EC00003220821D8E7B5F81530ADF80830002BBB
:106ED0000CBF07230623E7E70923E5E70322CBE7F7
:106EE000A8DF7047AADF70472DE9F04180468EB0D9
:106EF00015461F460E4611B9084600F09FFD15B90C
:106F0000284600F09BFD1C220DEB02000021FDF73E
:106F100009FA9DF81C30ADF80480002443F0020308
:106F20008DF81C3021460123032268468DF8063077
:106F3000CDE90A44CDE90C440894FDF7F3F93B7818
:106F40008DF800307B788DF801309DF8023023F009
:106F50001F0343F002032146142202A88DF80230D9
:106F6000FDF7E0F90A48CDF80CD001AB029302AA74
:106F7000149B0088ADF8105007A9ADF81240ADF889
:106F800014500696FFF7AEFF0EB0BDE8F08100BFCB
:106F9000F89A002030B587B041F60A032B4AADF8C5
:106FA0000C30044603A901208DF80E00FFF798FF6E
:106FB0000546D8B92288E2B922894AB1244B009308
:106FC000E16804F13C0342F62420FFF78DFFD8B9B5
:106FD000228C4AB11F4B0093616A04F13C0342F6D4
:106FE0002620FFF781FF78B9A36B7BB9284607B04D
:106FF00030BD194B0093616804F13C0342F629202F
:10700000FFF772FF0028D7D00546EFE71A788DF812
:1070100010205A888DF81120120A8DF812209A88B3
:10702000DB888DF815301B0A8DF813208DF816308B
:10703000120A0A4B8DF814200093072204F13C0336
:1070400004A942F65020FFF74FFFDDE7F89A002031
:10705000E89A0020D89A0020E09A0020F09A0020B8
:1070600029DF704728DF7047064B182202FB0030EB
:1070700000230422C0E90423037183608361C36099
:10708000704700BF0C9B002023B502460846C96824
:1070900043680093044B53F82150436910F80C1BCC
:1070A000A84702B020BD00BFFC9A002038B5194C9B
:1070B0002378182202FB03431A795869012A03D066
:1070C000032A1AD00F2038BD134A996915689A68A7
:1070D000DB68A2EB0532B2F5805F184401EB0531A5
:1070E00000EB053034BF92084FF48062FFF7B8FF21
:1070F0000028E8D10123A370E5E74FF080531B6916
:107100009BB2B0FBF3F0044B1B681844FFF7AAFFD7
:10711000EEE700BF0C9B0020049C002070B5134DCF
:107120006C780A2C1FD02E783444E4B2092C84BF2A
:107130000A3CE4B2182606FB0454A261207103C97C
:10714000A360049BE360AB7804F1100282E80300C3
:1071500023B100206B7801336B7070BDFFF7A6FF81
:107160001128F7D1F5E70420F7E700BF0C9B0020BA
:1071700070B5234CA3782BB100260228A67002D04C
:10718000032833D070BD25781E4A182101FB054124
:10719000136889680133B1EB033F136014D8637837
:1071A0001660013B63706B1CDBB21821092B01FBDD
:1071B000054188BFA5F10903002004312370FFF7C2
:1071C00063FF2846FFF750FF6378002BDAD0A378DF
:1071D000002BD7D1FFF76AFF0028D3D01128D1D0D8
:1071E0002178182303FB0141043105E0217818239D
:1071F00003FB014104310D20BDE87040FFF744BF9F
:107200000C9B0020049C002008B50A4B002119604B
:10721000094B1980997008460131FFF725FF0A29AB
:10722000F9D1064B00201860054BC3E90000C3E903
:10723000020008BD049C00200C9B0020009C002044
:10724000FC9A0020064A03461068042807D008600C
:10725000411C11601A68034B43F82020002070473E
:10726000009C0020FC9A002013B5CC180C43A40706
:1072700008D1009313460A4601460120FFF74EFF4E
:1072800002B010BD1020FBE707B500220B460092AC
:1072900001460320FFF742FF03B05DF804FB000046
:1072A000094B5A7899780132D2B2914208BF002234
:1072B000197891421FBF02705878182202FB0030E3
:1072C00014BF043000207047089C0020082910B526
:1072D000044602D0002000F0B1FBD4E90030BDE844
:1072E0001040184773B5054600240DF107000E46FF
:1072F0008DF8074000F0B0FB0DF10600FFF7D0FF5E
:1073000090B10670094B9DF8062045605A709DF8B3
:10731000070000F0C5FB24B9054B4FF48012C3F8F9
:107320000021204602B070BD0424F0E7089C002034
:1073300000E100E0204B21491A682F2300BF00BF65
:1073400000BF00BF00BF00BF00BF00BF8A422FD0F8
:1073500000BF00BF00BF00BF00BF00BF00BF00BF35
:1073600000BF00BF00BF00BF00BF00BF00BF00BF25
:1073700000BF00BF00BF00BF00BF00BF00BF00BF15
:1073800000BF00BF00BF00BF00BF00BF00BF00BF05
:1073900000BF00BF00BF00BF00BF00BF00BF00BFF5
:1073A00000BF00BF00BF00BF00BF00BF00BF00BFE5
:1073B000013BC3D1704700BF348400200024F40097
:1073C0000C4B0D484FF4003210B5C3F88020012457
:1073D0004FF48033C0F84833C0F808334460FFF7F7
:1073E000A9FF064B846000201860FFF7A3FF044B41
:1073F000187010BD00E100E000100140249D002045
:10740000159D00202DE9F3412549264B0025C1F8A3
:107410004051C1F84451C1F84851C1F84C51C1F82C
:107420000051C1F804511B68002B34D0D1F8044539
:107430001D49DFF888800968641A24F07F442F46CC
:107440001968A14212D81A7CDE69641A0D4462B12F
:107450005A691F7400929B6901934246082168464D
:1074600000F056FA08B100F0E9FABEB90F4A104B25
:1074700011781B788B4205D10133DBB2022B08BF98
:107480000023137012780B4B43F822500A4B4FF431
:107490008012C3F8002102B0BDE8F0813346CFE787
:1074A00000100140289D0020249D0020219D0020E7
:1074B000209D0020189D002000E100E0CD720F000B
:1074C0002DE9F74FA84AA94913780978A84C9942A1
:1074D0003BD00133DBB2022B08BF00231370A54958
:1074E0001278A54B0F6853F822003B1823F07F4316
:1074F00000220B60236815461646944613B942B124
:10750000236006E0196881420DD902B12360091A8F
:10751000196001262368DFF8689200930027BDB93F
:10752000DFF868A268E0401A0E44D968D3F81CE07E
:10753000C3F800C031B1BA1922F07F42C3E901217A
:10754000DD611D4673460122D8E700252E46E1E79E
:107550002846ED69874BD0F804C01B68DFF830E29D
:107560008168ACEB030222F07F42724500F2AD80ED
:107570000A4402600122027422680023C0E9013338
:10758000C361002A40F0AB802060C8E75A1C9AF81B
:107590000210D4F800B0D2B291428AF8002004BFA1
:1075A00000228AF80020182202FB03A31A799868A7
:1075B000022A77D0032A00F08580012A1CD190F896
:1075C00010C0BCF1000F17D1D96841601A69826000
:1075D0005A69C2609B698361684B1B78002B18BF96
:1075E00061464160B6E7904200F09E809046D269C5
:1075F000002AF8D1002303749AF800309AF8012089
:107600009A42C3D1236827B9009A9A4201D1002E29
:1076100042D0002B00F08580D3F80090584C554B99
:10762000D4F804651868574F351A3B7825F07F4524
:1076300003359BB94FF48033C4F84433C4F80433A2
:10764000514B4FF400324FF00108C3F880211A600B
:10765000C4F80080FFF76EFE87F80080A9452CBFB4
:107660004844401920F07F40C4F84005D4F8043560
:107670009B1B23F07F43801B033320F07F4083421A
:107680000AD9D4F80435C4F84035FFF753FE3E4B11
:107690004FF40032C3F80021384B00221A7003B0B7
:1076A000BDE8F08F5A46D846A2E78BF81020DBF8E9
:1076B0001CB00123BBF1000FF7D1002B9CD0C4F804
:1076C00000B099E700231A46F4E7A3EB0C0323F07C
:1076D0007F438B4234BFCB1A002303604AE7016823
:1076E000136899421BD85B1A1360C2614CE7A1EB87
:1076F0000C01D3F81CC01A46BCF1000F0AD0634637
:10770000D3F800C08C45F2D3ACEB010CC3F800C039
:107710009C4613460160C0F81CC0D861FFE61346C2
:10772000EEE7FFF74DFEB7E7404510D1DBF81C3020
:10773000236063B9DFF83CE001920121C9F8081029
:10774000CEF800300D4B1970FFF7F4FD019A136865
:10775000D269C8F81C2012B111680B441360236869
:107760005B4518BF012745E7209D0020219D002093
:10777000289D0020249D0020189D0020149D00209D
:1077800000100140159D002000E100E0089C002051
:10779000FEFF7F0008B5FFF713FE104B00200B2201
:1077A00018809A700E4B18600E4B18700E4B1870A4
:1077B0000E4B4FF48012E021C3F8802183F814139C
:1077C0001A6002F18042A2F56F22C2F8080583F820
:1077D0001113074BD2F804251A6008BD089C00203D
:1077E000289D0020209D0020219D002000E100E038
:1077F000249D0020074B9B784BB132B128B1036820
:10780000187C20B959745A617047072070470820C6
:10781000704700BF089C00202DE9F743DFF8848003
:1078200098F8023005460E461746ABB3A0B30429BC
:1078300030D9436983B3437C0024012B0DF1070049
:107840000CBF8946A1468DF8074000F005F90DF1FF
:107850000600FFF725FDD8B1012303700F4B4560EB
:10786000D3F80435C0E90497C0E902369DF8063024
:1078700088F801309DF8070000F012F924B9084B90
:107880004FF48012C3F80021204603B0BDE8F08316
:107890000424EFE70724F7E70824F5E70010014088
:1078A00000E100E0089C0020064A92783AB130B12D
:1078B000426922B1002202740221FFF713BD0820A1
:1078C000704700BF089C00204B1C30B5DB0004460D
:1078D00012F003009BB20DD1074D2A601A44074BEA
:1078E0001A60074B1870074B1870074B1C80074B2A
:1078F000198030BD0720FCE7349D0020309D00201A
:107900002C9D00203C9D0020389D00203A9D0020A9
:107910002DE9F347DFF8C080B8F800308B42064607
:107920000D4617464CD300240DF107008DF8074093
:1079300000F092F8244B254A25481B78008892F8DD
:1079400000C084455FFA8CF138BF4C1CDBB238BFF5
:10795000E4B2A3422ED014781178CBB2884286BF0D
:107960000133DBB2002313709DF8070000F098F894
:107970004FF6FF739C4225D0DFF86090D9F80020C5
:107980004FEAC40A42F8347002EBC403AEB1A5B1A9
:10799000104BB8F800001B682A4604FB0030314643
:1079A00003F0F0FBD9F80030534400209D8002B072
:1079B000BDE8F0874FF6FF74D6E700209880F6E721
:1079C0000920F4E70420F2E73C9D00202C9D0020D4
:1079D0003A9D0020309D0020389D0020349D0020DD
:1079E00070B5104C104D22782B789A4200D170BDA2
:1079F0000E480F4A2378126806880E4802EBC3012E
:107A0000006852F83320898803FB060090470A4932
:107A100022780988D3B2914286BF0133DBB20023BA
:107A20002370E0E73C9D00202C9D0020389D002025
:107A3000349D0020309D00203A9D00201FB500217C
:107A4000CDE9021001AA44F20100ADF80410FCF7E0
:107A5000A8FE05B05DF804FB70B5EFF3108672B6B2
:107A60000C4A946801239CB993600B4B0B4DD3F8DF
:107A7000801029401160C3F88050D3F88410516001
:107A80004FF0FF32C3F88420047006B962B670BDAF
:107A90000370FAE7409D002000E100E0FC06FFBD16
:107AA00010B5084B9A685AB150B9EFF3108172B60D
:107AB000054A1C6814605C685460986001B962B63D
:107AC00010BD00BF409D002000E100E003462AB148
:107AD00010881A4619448A4203D170474FF6FF7046
:107AE000F7E712F8013B40BA80B25840C0F30313E5
:107AF000584080EA0033580100F4FF509BB25840D0
:107B0000E9E70000064B074A00201870064B1A6090
:107B10000822C3E90120C3E90300C3E90500704757
:107B20004C9D0020509D002030B000200020704768
:107B300030B5F9B1124B5C6800220A60E4B1B0F5CF
:107B4000167F1BD8D868013C01305C60D8601C6887
:107B500018694FF4177505FB00440C60012101FA08
:107B600000F49969013000F0070021431861996120
:107B7000104630BD0E20FCE70420FAE70C20F8E7A1
:107B800030B00020F0B51C498A689AB34D690E6880
:107B9000AC1A04F0070423464FF4177707FB036C75
:107BA000604511D1012000FA03F5886968408861B9
:107BB00000204E68D1F818C04FF0010E7344002524
:107BC000164403F007030AE0013303F007039D4264
:107BD000E4D11020EDE74AB1013A1C4601250EFA26
:107BE00004F414EA0C0FA6EB0207F4D00DB1C1E9BE
:107BF0000172F0BD0420FCE730B00020064A136992
:107C00001268013B4FF4177103F0070301FB0323D4
:107C1000C3F858020020704730B0002030B5C0B122
:107C2000B9B10E4BDA68B2B1013ADA609A681C68F1
:107C300001329A605A694FF4177505FB02440460DB
:107C40000132D4F85802086002F007025A6100209D
:107C500030BD0E20FCE70420FAE700BF30B0002062
:107C60003FB40C49086890B10B4B1C687CB10B4ABF
:107C70001568CDE9025000238DF804300B601360C5
:107C800004AB13E90700234604B030BC184704B026
:107C900030BC704754B0002058B0002064B00020C1
:107CA000DC2810B509D0DD2810D0C02816D1FFF788
:107CB000D7FF0E4B0E4A1A6010BD0E4A0E4B1968C4
:107CC0001368581C1060C022CA54F2E7094A0A4BD4
:107CD00019681368581C1060DB22F5E7064B054A4B
:107CE000196813685C1CC8541460E2E740840020E3
:107CF000117D0F0054B0002064B00020C02802BFE6
:107D0000014B024A1A60704740840020117D0F0029
:107D1000C02810B409D0DB280BD0094B094A1968D8
:107D200013685C1CC854146006E05DF8044BFFF750
:107D300097BF054B054A1A605DF8044B704700BFBA
:107D400064B0002054B0002040840020A17C0F00CB
:107D500007B501228DF807000DF10701002002F0A0
:107D6000C7FC00280CBF0420002003B05DF804FB12
:107D700010B5064A064C12682368D05CFFF7E8FF8E
:107D800010B923680133236010BD00BF68B0002024
:107D90005CB0002008B5C020FFF7DAFF28B9034B1C
:107DA0001B6813B9024B034A1A6008BD5CB000207F
:107DB00044840020717D0F0008B5DB20FFF7C8FF69
:107DC00010B9024B024A1A6008BD00BF448400206B
:107DD000D57D0F0010B50C4A0C4C12682368D35C9B
:107DE000C02B03D0DB2B0DD0042010BDDC20FFF70F
:107DF000AFFF0028F9D12368054A01332360054B02
:107E00001A60F2E7DD20F2E768B000205CB00020E5
:107E1000717D0F00448400207FB5184C184D194E19
:107E2000002002F005FC30B322689AB1296833685B
:107E300099420FD2012201A9002002F005FC10B9DD
:107E40004FF0FF3001E09DF804000F4BC0B21B68FB
:107E50009847E5E70D4B1B686BB10292084A022177
:107E6000126803928DF8041004AA12E9070004B006
:107E7000BDE87040184704B070BD00BF64B000207A
:107E800054B0002050B000204084002058B00020A2
:107E9000014B18600020704758B00020034B1A783F
:107EA0000AB901221A700020704700BF4CB00020B0
:107EB000014B0020187070474CB000202DE9F04FA6
:107EC00085B0002851D02A4F3B78012B07D0022BD8
:107ED00014BF08240424204605B0BDE8F08F254DCA
:107EE000DFF8A090244E254CDFF89C80DFF89CA0A2
:107EF000DFF89CB0C9F8001000232B60022330602B
:107F00003B70C4F800802A68D9F800309A4215D333
:107F1000C4F80080FFF73EFF044608BB184B1B68FF
:107F200001223A70E3B18DF80420326802922A6887
:107F3000039204AA12E907009847CCE733682A683D
:107F40009A5CC02A03D02A689B5CDB2B04D123688F
:107F5000534508BFC4F800B023689847042801D1EE
:107F60000024B8E71128CED1FAE71024B3E700BF08
:107F70004CB000205CB0002068B000204484002099
:107F800058B0002060B00020957D0F00717D0F007B
:107F9000B97D0F00054B064A1860064B1960064B69
:107FA00000201860054B1A60704700BF64B00020C5
:107FB000FD7C0F0050B0002054B000204084002011
:107FC000064B07481B68DB00DBB2002203705B42F4
:107FD00042708270C3700421FFF770BF94B000201C
:107FE0006CB0002070B52B4C2B4D02462378012B32
:107FF00014D0022B21D0002B4BD1002A49D1274885
:10800000FFF752FC08B1FFF719FD254B1B68002B49
:108010003FD0244ABDE8704010781847012A38D173
:108020002968214B06311868FFF748FF08B1FFF7B0
:1080300005FD022323700022D8E7022A16D0032A66
:108040000CD032BB194B15481A6041F67F21FFF75F
:10805000E3FBF0B1BDE87040FFF7F0BC144A1368D1
:10806000013303F0070313600023E3E70F4A1368AB
:10807000052B0AD001331360074B19680A4BBDE882
:10808000704018680631FFF719BF064B01221A70BD
:10809000EAE770BDB8B00020ACB0002070B000209E
:1080A000A8B00020B0B00020C0B00020B4B00020C4
:1080B00098B00020F0B585B004AB03E907009DF847
:1080C0000400032874D8DFE800F00802A3A601200A
:1080D00005B0BDE8F040FFF785BF039E544C032E6A
:1080E00040F28280029D6B7813F00F0265D00E2A59
:1080F0007AD1042E55D02A78500652D5110650D583
:108100001A44AB781A44EB781A4412F0FF0248D1B3
:10811000B71E39462846FFF7D9FCEB5B834240D1B6
:1081200044492A780B6802F00702D8B282422BD168
:10813000013303F007030B60FFF742FF3E4B0122C0
:1081400030461A70FFF75AFD08B1FFF777FC38493F
:108150004FF41670FFF7ECFC002862D0042802D020
:108160000020FFF76BFC35480521FFF713FF08B12E
:10817000FFF764FC324B1B68002B56D04FF0000019
:1081800005B0BDE8F040184720684FF41671FFF7BE
:1081900001FF08B1FFF752FC05B0BDE8F040FFF762
:1081A0000FBF20684FF41671FFF7F4FE00283CD093
:1081B00005B0BDE8F040FFF741BC2978AA780B4430
:1081C0001344EA78134413F0FF030DD11D4A1268DB
:1081D0000132C1F3C20102F00702914204D11A4AEE
:1081E00003201370FFF7FEFE25681DB14FF41671D2
:1081F0002846D9E70E494FF41670FFF799FC60B195
:10820000042802D02846FFF719FC0C480521CBE7CB
:108210000A480521C8E70320CAE720684FF4167111
:10822000C2E720684FF416719FE705B0F0BD00BFAC
:10823000BCB0002094B0002090B000209CB0002082
:10824000A4B0002098B00020B0B000200220FFF7BA
:10825000C9BE0000074B10B5044618600648FFF77A
:1082600017FE08B1FFF7EAFB002C0CBF0E20002020
:1082700010BD00BFA4B00020B5800F00184A1948F7
:10828000002310B51360184A1360184A1360184A87
:108290001370184A1370184B184A01211960184BB3
:1082A0001960184B1970FFF7A5FA08B1032010BD2B
:1082B000FFF728FC0028FAD1FFF7F0FD0028F6D1DF
:1082C000114C4FF416702146FFF732FC0028EDD117
:1082D00020684FF41671BDE81040FFF75BBE00BF89
:1082E000C0B000202CB60F00ACB00020B4B000200D
:1082F00090B00020B8B0002094B000204D820F0054
:1083000098B00020B0B00020BCB000200C4A08B5E6
:10831000002313600B4A1360FFF708FC08B1FFF756
:108320008DFBFFF7C5FD08B1FFF788FB0648FFF797
:10833000BBFA042802D10020FFF780FB002008BD13
:10834000A8B00020A4B0002070B0002037B50D46C2
:10835000044698B191B10A4B19780022019259B1A3
:1083600001A91A70FFF75AFC019B063B2B8023687A
:108370000433236003B030BD0420FBE70E20F9E78F
:1083800090B000200438FFF7FDBB18DF70470000F5
:10839000F0B51D46154B87B018680F4659681B7A13
:1083A00003AC03C42370124B18685968114B009337
:1083B00001AC03C42046164602F01BFF21460246CC
:1083C000384602F0DFFE01A802F013FF01A90246C1
:1083D000304602F0D7FE684602F00BFF69460246BF
:1083E000284602F0CFFE07B0F0BD00BF30B60F0048
:1083F00039B60F00312E30000120704710B51C46F1
:108400000B781E2B0AD000232022052102F088FBC6
:108410004FF6FF70A04228BF204610BD0020F9E7AC
:10842000F8B5069F14460D463A46002118461E46EA
:10843000FBF778FF7CB14FF0E023D3F8F03DDB078A
:1084400000D500BE4FF0FF300AE0284600F0F6F9F4
:10845000013504F50074BC4206EB0401F5D3204657
:10846000F8BD0000F8B50A4F0D461E460024069BD5
:108470009C4206EB040101D32046F8BD3A4628464B
:1084800000F0B2FA0028F7D0013504F50074EEE7E9
:10849000C4B0002030B5264D2A7A8DB09AB107AC11
:1084A0001422002120460625FBF73CFF8DF81C50C6
:1084B0000B9B009394E80F00FCF7C6FF0620FCF727
:1084C000F1FC0DB030BD2B68002BFAD0194B197898
:1084D00019B105201A70FCF7E5FCD5E900329A4283
:1084E000EFD307AC142200212046FBF71BFF6B7A69
:1084F000DBB106234FF420424FF474214FF4602087
:108500008DF81C3002F02EFE0028D1D01022002160
:1085100003A8FBF707FF4FF460224FF4205303A892
:10852000CDE90423FFF731FFC2E78DF81C30BFE728
:10853000C4B0002048840020024B0B604FF400734D
:1085400013807047090101000120704700487047FF
:10855000F6840020044B054A1878054B002814BF08
:1085600010461846704700BFE0B20020AB840020E0
:10857000498400202DE9FF411E4B187020B11E4B8D
:108580002A229A720022DA721C4A1D4DDFF878C046
:1085900017461C4BEE4603F11006744618685968DE
:1085A000F046A8E803000833B342C646F6D12B785C
:1085B00003F00F0310336B4413F8103CD373114BCB
:1085C00018685968A646AEE803000833B3427446FB
:1085D000F6D115F8013B04A901EB1313654513F817
:1085E000103C9373A2F10202D3D100233B7404B078
:1085F000BDE8F081E0B20020F684002064B30020E2
:108600006000001041B60F006800001010B570B98E
:10861000134B14481968022202F0B4FD0123013300
:10862000DBB211485B0043F44073038010BD0528A2
:1086300014D80B4B53F82040204602F0DAFDC3B2A9
:108640001F2B28BF1F23084A2046E118884202F149
:108650000202E4D010F8014B1480F7E70020E5E7B0
:1086600008850020E4B20020E2B200204DDF704710
:108670004EDF70474FDF704750DF704712DF7047A3
:10868000002000F0DBBC00001FB5244B402283F823
:10869000272300238DF807304FF4405304465A68CF
:1086A0001F4B9A4227D10DF10700FFF7E7FF9DF816
:1086B000073003B30120FFF7DBFF0120FFF7D6FFF0
:1086C0000120FFF7D7FF02A8FFF7D6FF029BDA07CA
:1086D00002D5002000F026FE029B9B0702D5022057
:1086E00000F020FE2046FFF745FF00F027F802F0DB
:1086F0000BFD04B010BD002301A88DF80430FCF779
:108700001FFC084B039303A8FCF742FCFCF746FC54
:108710004FF08043D3F838340293D7E700E100E00C
:10872000DBE5B15125930F00012000F0FBBD0120D6
:10873000FCF7B8BB0220FCF7B5BB00007FB52F49A2
:108740002F4802F047FD4FF440532E4A596891429A
:108750004CD11A78102A46D9142A186944D95B6971
:10876000294CB3FBF4F50A2201A904FB153402F0ED
:108770008BFD2649224802F02DFD01A9204802F078
:1087800029FD23491E4802F025FD0A2201A9284699
:1087900002F07AFD01A91A4802F01CFD1D49184893
:1087A00002F018FD4FF47A760A2201A9B4FBF6F51F
:1087B000284602F069FD01A9114802F00BFD154998
:1087C0000F4802F007FD0A2201A906FB154002F03E
:1087D0005BFD01A90A4802F0FDFC0F49084802F0C0
:1087E000F9FC04B070BD00200023B9E70B49044830
:1087F00004B0BDE8704002F0EDBC00BF5FB60F00F2
:1088000020850020DBE5B15140420F006CB60F001F
:108810006AB60F006EB60F0079B60F0070B60F0083
:1088200010B503461C1A944200DB10BD0C781CB135
:10883000013103F8014BF5E72024FAE72DE9F34174
:108840000C4605464FF4007200212046FBF76AFDF6
:108850006DB95E493E22204602F094FC552384F80F
:10886000FE31AA2384F8FF3102B0BDE8F081B5F5EE
:10887000017F2DD8691EB1F5817F24BF6FF4817807
:1088800005EB0801C9B10B02C1EBC15103F58070C2
:1088900004EB412440F693651A1FB2F5696F03F1AA
:1088A000010206D2AB4214BF91B24FF6FF7124F819
:1088B000131090421346EFD1D6E7F823237004F14A
:1088C00009022346FF2003F8010F9342FBD1DAE7A8
:1088D000B5F5027F3BD86FF4017C65443DB9204675
:1088E0003B490B22FFF79CFF2823E37220343949D0
:1088F0002E014FF0000801EB05256FF01D07022E39
:10890000B2D80B2229462046FFF78AFF53237E2246
:1089100060216374E3746376B31C84F80D80A773DD
:10892000E1732274A27484F8148084F81580A7750A
:10893000E17522766383E86830B102F05AFCE061A9
:10894000013620341035DAE74FF4E910F7E7224B0F
:108950009D4289D86FF40277EA19012A0FD81D4B7E
:1089600003EB0213D9680191084602F042FC019919
:108970000246204602B0BDE8F04102F003BC6FF4AD
:10898000FD76A9190902B1F5801FBFF46DAF134B35
:10899000236003F1144303F52C1303F602336360E1
:1089A0000F4BC4F8FC314FF46963A3614FF40053DB
:1089B000A5F20B254FF48072A3600A4B6561E1605C
:1089C0002261E36104F12000D4E700BF7CB60F0010
:1089D000A7B60F0048B70F00080101005546320A3C
:1089E000306FB10A29009A23F7B5654B14460A681F
:1089F0009A420D4639D103F114434A6803F52C130A
:108A000003F602339A4230D1D1F8FC215D4B9A42F1
:108A10002BD18B6823F4FF5323F01E039B049B0C84
:108A2000B3F5005F21D10B69B3F5807F1DD1C86814
:108A300010F0FF0619D1CB69534A934205D0534A2F
:108A4000934215D0524A93420FD1A0F58053B3F50B
:108A5000692F07D201234FF4807205F12001FBF743
:108A600049FE22E0B0F5805F1FD34FF0FF3021E0D8
:108A700001276772CB68B3F1102F1DD10422343166
:108A8000684602F07FFB042205F138010DEB02007D
:108A900002F078FB009BB3F5742F03D1019BB3F573
:108AA0007E2F01D02772E0E7A772AB69002B37D188
:108AB0004FF4007003B0F0BDA3F57422B2F5204F5F
:108AC00028D2E27A01F12007DAB9324A934218D368
:108AD0002B69B34215D90422B919684602F052FB3A
:108AE000009BD02B14D10422311D0DEB0200394420
:108AF00002F048FB264B019A9A424FF001030DD138
:108B0000E372E8682A6901233946A0F5A030A6E798
:108B10000836DDE7B3F5805FC7D301232372A4E7EE
:108B20002268934207D041F263018B4200D80AB118
:108B30004FF0FF3323606B6941F263029342B7D871
:108B400003F0070204EBD303012191401A7B114289
:108B5000C8B204D16168024301311A736160D4E97B
:108B600000329A42A4D30120FBF7A6FD637A002BC2
:108B70009ED0A37A002B9BD10123237298E700BFDC
:108B80005546320A306FB10A4028A5AD3C8263D603
:108B900029009A2300D80F004FF08053D3F83001FA
:108BA000082802D1D3F8343123B9A0F10D0358427B
:108BB000584170470120704742DF704743DF7047DC
:108BC00044DF704712DF704770B4234C94F8D830FC
:108BD0008BB3224B5B68C3F308032BB1014670BC17
:108BE0001F48012201F030B8EFF310828ABB1D4B01
:108BF0005A68C2F3C01312062BD594F8D830002B54
:108C0000FBD118E0D6F82C31D6F8502100211344BE
:108C10008A0002F1804202F51C320131D2F808517B
:108C2000D2F8302108292A441344F1D194F8D820ED
:108C3000DBB29A42E6D894F8D8300133DBB284F83C
:108C4000D83001230360BFF36F8FBFF34F8F70BC29
:108C50007047054EEAE700BF78B3002000ED00E062
:108C6000C98B0F0000E100E000700240082870B5D9
:108C7000184B194E044618D1D3F8C054EA0327D430
:108C8000D6F8C0201548C3F8A027C3F8A457FFF7AB
:108C90009BFF18204443321933592B443351D38856
:108CA00015FA83F5ADB2D58070BD00F5947214212C
:108CB00053F822501822424301FB00330848B258AF
:108CC000C3F80027EDB2C3F8045700EB8400DEE7D9
:108CD0000025DEE70070024078B3002048700240B3
:108CE0002870024010B41049182303FB00114A8A6F
:108CF0000B8ACC689B1A8A8A9BB2934228BF134680
:108D00001422424302F1804202F51C32C2F80046AE
:108D1000C2F804362344CB60044B5DF8044B03EBEC
:108D20008000FFF751BF00BF78B3002004700240FD
:108D300007B54FF4405300205A68084B9A420AD1B5
:108D40008DF807000DF10700FFF73CFF9DF80700C5
:108D5000003818BF012003B05DF804FBDBE5B1511A
:108D600007B5FFF7E5FF58B1002301A80193FFF70E
:108D700027FF0198003818BF012003B05DF804FBFD
:108D80004FF08043D3F80C0400F00110A0F1011360
:108D900058425841F1E7000008B5FFF715FF054AB2
:108DA00092F8D8302BB192F8D830013BDBB282F880
:108DB000D83008BD78B3002070470000014B8022F6
:108DC0005A60704700E100E0024B8022C3F8842023
:108DD000704700BF00E100E0074BD3F80014D3F860
:108DE00000240A43C3F800240022C3F858214FF49A
:108DF0008002C3F8042370470070024070B58A787F
:108E00004E793E4C02F07F0318200C25D2095843BE
:108E100005FB02000D79204406F0070645EA062509
:108E20000581C97801F00301012922D001203449CC
:108E300000FA03F49AB903F10C05A840C1F8040341
:108E4000D1F8140503F594732043C1F8140541F8D3
:108E50002320BFF36F8FBFF34F8F012014E0023345
:108E60009840C1F80403D1F810352343C1F81035F8
:108E7000EFE7082B09D04FF0E023D3F8F00D10F006
:108E8000010001D000BE002070BD1D4BDAB9B4F85E
:108E9000D42012B18022C3F81C250022C3F850212F
:108EA000D3F8002312F4001208BFC3F85421144B66
:108EB0004FF44012C3F80423D3F8142542F480720F
:108EC000C3F81425C5E70022C3F82C21B4F8C82044
:108ED00012B18022C3F81C25094BD3F8002312F4E9
:108EE000001208BFC3F85421064AC3F80423D3F87C
:108EF000102542F48072C3F81025AAE778B3002049
:108F00000070024000082000F7B51F4601F07F0006
:108F100018231F4CCD090E4643430C2101FB05319C
:108F200004EB010C62500022ACF80470ACF806208F
:108F300018B1F5B1FFF7D6FE18E017BB154BD3F803
:108F40008034C3F3C0139D421BD01348FFF724FFA6
:108F5000124B5B68C3F30803003B18BF0123009367
:108F60003A463B463146384600F059FE012003B0F0
:108F7000F0BD1C44A37A002BF8D0A572FFF776FE53
:108F8000F4E7002DD6D10648FFF706FFEEE700BF55
:108F900078B30020007002405070024000ED00E005
:108FA0004C70024011F07F0307D1084B01225A6533
:108FB000BFF36F8FBFF34F8F7047082B1EBF034B5C
:108FC00041F48071C3F81815F2E700BF0070024049
:108FD00011F0770F10D0094B41F48072C3F81815C7
:108FE000C3F80C25CA0904BF01F5947143F8212088
:108FF000BFF36F8FBFF34F8F704700BF0070024009
:1090000010B500221146930003F1804303F51C3391
:109010000132082A59609962F5D1064B064C596213
:10902000DC22996420460021FBF77CF94023A382CF
:10903000238110BD0070024078B300202DE9F04F6D
:10904000B14BB24AD3F80013002385B01C4601206F
:109050001D4621FA03F6F6070BD552F8236046B1F8
:1090600000FA03F6344342F82350BFF36F8FBFF387
:109070004F8F0133192BECD1E30706D5FFF7C0FF63
:1090800000210122084600F0A1FD14F4006FA04D5C
:1090900008D09D4BD3F8A8369BB2A5F8D230012357
:1090A00085F8D730A7021BD5974BD3F81435DE05CA
:1090B00002D50820FFF7DAFD95F8D7305BB1B5F897
:1090C000D2200023012185F8D73092B200911846B2
:1090D000882100F0A4FD01220321002000F066FD9C
:1090E000600217D5884FD7F8006406F44073F10585
:1090F000C7F8003407D501220421002000F056FDF6
:109100000123C7F82C35B20504D501220521002022
:1091100000F04CFD23022BD57B4BD3F88014C9B251
:109120008DF80810D3F88424D2B28DF80920D3F832
:1091300088048DF80A00D3F88C048DF80B00D3F85E
:1091400090048DF80C00D3F894048DF80D00D3F83A
:1091500098048DF80E00D3F89C348DF80F304F062C
:1091600001D1052A04D0012202A9002000F041FD0E
:10917000684B23405BB195F8D830002B40F09C80C1
:109180004FF0E023D3F8F03DDE0700D500BE604F7E
:10919000DFF874A1DFF88491DFF884B1B8460026C7
:1091A00006F10C0324FA03F3D807F1B21FD51423F8
:1091B00003FB06A3082ED3F80837DBB200F0848047
:1091C000B8F808209A427FD1182303FB0653B8F859
:1091D0000420DB889BB29A4276D941B995F8D83001
:1091E000002B6DD001224946584600F02DFD013676
:1091F000092E08F11808D3D1474B2340002B58D033
:10920000414BD3F86C84C3F86C84BFF36F8FBFF30A
:109210004F8F14F4806407D0D3F88044D3F880349F
:109220001906C4F3C0145ED54FF0000ADFF8E090D1
:1092300000264FF0180B28FA06F3DA07F0B201D433
:10924000AEB9A4B1304B142202FB06330BFB06521D
:10925000D3F80416538A11FA83F39BB25382538ACC
:10926000B9F810109BB2994240D9FFF73BFD013687
:10927000082E09F11809DED1002418264FF0010943
:1092800004F1100328FA03F3DB07E0B203D45CB95E
:10929000BAF1000F08D006FB0452B988D3889BB2FC
:1092A00099422ED9FFF7E2FC0134082C07F1180788
:1092B000E6D105B0BDE8F08F002385F8D83066E729
:1092C0004846FFF769FD92E7182303FB0653DA8847
:1092D000A8F80420DA8801230093002392B21846EC
:1092E00000F09DFC83E74FF0010A9FE7528A0123BB
:1092F0000093002340F0800192B2184600F08FFCEA
:10930000B5E782F80A90CFE7007002400071024092
:1093100078B30020FCFB1F00000400014C700240E9
:10932000998D0F00012813B5044600F0BF80022874
:1093300055D0002851D1764BD3F80025002A4CD1C6
:109340004FF40062C3F80024BFF36F8FBFF34F8F59
:10935000FFF722FC60B16F4BD3F8001C032269BBFE
:1093600049F27531C3F8001CC3F8142DC3F8001C72
:109370004FF08053D3F83031082B0CD1654BD3F824
:10938000001CC022E9B949F27531C3F8001CC3F8CA
:10939000142CC3F8001C5E4B0124C3F80045BFF336
:1093A0006F8FBFF34F8FFFF7DBFCB0B9FFF7C0FC47
:1093B00050B102B0BDE81040FFF7FEBBC3F8142D5A
:1093C000D6E7C3F8142CE6E74FF08043C3F800015A
:1093D000D3F800210192019A1C6002B010BD4C4CE0
:1093E000D4F804351BB1FFF7BBFC0028F5D1D4F845
:1093F00000341B05FBD54FF40063C4F80034BFF301
:109400006F8FBFF34F8F4FF08053D3F83031082B5D
:109410000CD1404BD3F8001C00293FD149F27532E2
:10942000C3F8002CC3F8141CC3F8002CFFF7B4FBDE
:1094300058B1384BD3F8001CA1BB49F27532C3F8C0
:10944000002CC3F8141DC3F8002C4FF08053D3F840
:109450003031082B2E4B0AD140F2E372C3F80028BA
:109460004022C3F80428BFF36F8FBFF34F8F8022D1
:109470002949C3F81C25C3F80413284BC3F88421D9
:109480005A60FFF76DFC0028FBD0214B0122C3F886
:109490000425BFF36F8FBFF34F8F9EE70022C3F801
:1094A000142CC3E70022C3F8142DCEE7184BD3F8D1
:1094B0000025002A91D00022C3F80425BFF36F8F46
:1094C000BFF34F8F15498020C1F88400D3F80013F3
:1094D000C3F80813C3F80025BFF36F8FBFF34F8F96
:1094E000FFF726FC78B1FFF769FB0D4B5A68C2F312
:1094F0000802003A18BF01220221002002B0BDE894
:10950000104000F053BB4FF080435C60EDE700BFBC
:109510000070024000E006400514800100E100E018
:1095200000ED00E00A44034690B2884202D39A89D3
:10953000824202D25A89104480B2704782888A429D
:1095400010B504D884898B1A9BB29C4203D24389FC
:109550001A44891A8BB2038210BD930813B501EB2C
:109560008303044699420BD112F0030206D0002374
:1095700001A8019301F006FE019B236002B010BD1B
:1095800051F8040B2060EDE72DE9F04385B0144657
:10959000BDF83050AB4238BF4289A3EB05091FFA32
:1095A00089F938BFA9EB0209828838BF1FFA89F907
:1095B0004A4588460746194605D2FFF7BFFF058A88
:1095C000B0F80490ADB2B9F1000F1FD0A14528BF8B
:1095D000A146BC88AC421DD9FA889DF83400396890
:1095E000661BA9EB04042C44B3B214FB02F416FB73
:1095F00002F60128B6B2A4B202FB051116D09945B5
:109600000BD802FB09F2404601F0BCFD484605B00C
:10961000BDE8F0832D1BADB2DCE73246404601F0D9
:10962000B1FD3968224608EB0600EDE7994506D8FA
:1096300019FB02F292B24046FFF78FFFE6E726F0F1
:109640000305ADB22A4640460191FFF786FF16F0AA
:10965000030628D001990D44C6F1040189B2A14244
:109660004FF0000328BF2146641A039303ABA4B252
:10967000A8191A4685420CD13B68013E164419448C
:109680008B420BD1039BC8F80030002CBED0224681
:10969000D1E715F801CB03F801CBEBE713F8012B69
:1096A00006F8012FECE73968EFE713B5930800EBF4
:1096B0008303984209D112F0030204D00B6801938E
:1096C00001A901F05FFD02B010BD0C6840F8044B29
:1096D000EFE770B59A42A2EB03041D4638BF4389F9
:1096E000A4B238BFE41A838838BFA4B2A3420E469E
:1096F000114602D2FFF722FF848874B18288AA4201
:1097000008D9C2880168304602FB051101F03AFD14
:10971000012070BDAD1AADB2F1E72046F9E72DE9A1
:10972000F0430746B0F80E908588048A1646C28832
:10973000007A85B01FFA89F9A4B288BBA145A9EBCC
:10974000040038BF7C8980B23CBF001B80B2281A5D
:1097500080B2864228BF06464C46AC4228D2A5EBD2
:109760000408751B386825441FFA88FC15FB02F5B0
:1097700018FB02F8012B1FFA88F8ADB202FB0400B7
:1097800022D0664517D8724301F0FCFC32464946A8
:109790003846FFF7C7FEF881304605B0BDE8F083D4
:1097A000AE4221BF761B02FB0611A1462E46D3E72F
:1097B000641BA4B2D1E74246009101F0E3FC00999A
:1097C00038682A464144DFE7664505D816FB02F2B1
:1097D00092B2FFF76AFFD9E728F00304A4B2224649
:1097E000CDE90001FFF761FF18F00308019929D0C6
:1097F000C8F104039BB2AB4200980A68039228BFE9
:109800002B46013CED1A0DF10C0C2044ADB2444640
:109810006246013C1CF801EB00F801EF14F0FF0474
:10982000F7D13868904408EB0304421EA04504D1E8
:109830001844002DAAD02A46CBE718F801CB02F82D
:1098400001CFF3E73868F4E7B2F5004F10D8828013
:109850005200C38092B29DF800300372531E838180
:1098600052420023C381016042810382012070477C
:1098700000207047C189028A89B292B29142A1EB5D
:10988000020338BF428980889BB23CBF9B1A9BB2BF
:10989000984228BF18467047C289038A92B29BB289
:1098A000D31A58425841704710B5C189028A84883A
:1098B00089B292B2914238BF4089A1EB02039BB2B8
:1098C0003CBF1B1A9BB2E01A80B210BD38B5C289EA
:1098D000038A04469BB292B2FFF7FBFE218A05463B
:1098E00082B289B22046FFF71DFE2082284638BD8D
:1098F00073B5C389058A0026ADB20446CDE900568A
:109900009BB2FFF741FE218A0546024689B22046F6
:10991000FFF708FE2082284602B070BD38B5C58921
:10992000028AADB292B2AA42A5EB020388BF428975
:109930009BB288BF9B1A828888BF9BB29A4204461A
:1099400014D1007A90B938BD9B1A9BB29342FBD2D6
:10995000E288206802FB030001F014FC0122294682
:109960002046FFF7DFFDE0810120ECE72B46EDE725
:1099700012B10023FFF7D3BE104670470023C38106
:10998000038283885B009BB25A1E5B4282814381C3
:109990000120704701720120704700000B4B63B13A
:1099A0000B4B1B78834206D90A4B1B6800EB400027
:1099B00003EBC0007047C01AC0B2012803D8064BA1
:1099C00000EB4000F4E70020704700BF00000000FB
:1099D00058B4002054B4002078B70F0070B5372277
:1099E000002105460E480F4EFAF79CFC1022FF217D
:1099F0000D48FAF797FC1222FF210C48FAF792FC67
:109A000000F076FD00242046FFF7C8FF4368284693
:109A1000984733780134E4B20133A342F3DA70BDDE
:109A200059B4002058B400205CB400206CB400206D
:109A300037B50C460546C868019200F061FDE36841
:109A4000019A0021284603B0BDE83040184773B59D
:109A5000054614463AB90378012B04D1104601910A
:109A6000FFF7B2F90199281DFFF758FF06462CB9F8
:109A70002B78012B02D12046FFF7A0F936B94FF021
:109A8000E023D3F8F03DDB0700D500BE02B070BD87
:109A9000024B5878003818BF0120704759B4002095
:109AA000024B1878C0F38000704700BF59B4002003
:109AB000014B1878704700BF90B40020F8B5164EDF
:109AC0003178054629BB154C15483722FAF72AFC90
:109AD000201DFFF753FF134B1C60134B23B113489A
:109AE000AFF30080124B1860104F00242046FFF7A0
:109AF00055FF036898473B780134E4B20133A34231
:109B0000F4DA2846FFF758F92846FFF757F90123FA
:109B100033700120F8BD00BF90B40020A086002063
:109B200059B4002094B400200000000058B4002074
:109B300054B4002010B44378023B0A46032B15D8D6
:109B4000DFE803F0022C1B23164B1978CC0725D530
:109B500019786FF300011970197800246FF341012F
:109B600019705C70197864F3820119700E4B5DF8FE
:109B7000044B01461868FFF76ABF0A4B1978C907FA
:109B80000CD5197841F00401EFE706490B78DB07A3
:109B900004D50B786FF382030B70E7E75DF8044B95
:109BA000704700BF59B4002094B400201FB50023B3
:109BB000CDE901338DF804008DF8051001A8114698
:109BC0000393FFF7B7FF05B05DF804FB1FB5002353
:109BD000CDE9013303938DF8040001238DF80810BB
:109BE00001A811468DF80530FFF7A4FF05B05DF818
:109BF00004FB1FB5144600230822CDE9013303936B
:109C00008DF8040006230DEB02008DF8053001F0FD
:109C1000B9FA214601A8FFF78DFF04B010BD1FB5AA
:109C20000024CDE901448DF8040007208DF80500DB
:109C30008DF8081001A89DF8181003928DF80930CE
:109C4000FFF778FF04B010BD1FB54FF40063CDE9F6
:109C50000130039101A81146FFF76CFF05B05DF8D4
:109C600004FB00008B7803F07F03082B08D94FF02A
:109C7000E023D3F8F03DDB0700D500BE002070479D
:109C80004A790B7902F0070243EA0223CA7802F00C
:109C90000302022A0ED0032A18D0012AEED10F4A5D
:109CA0009278022A40F2FF3208BF4FF480629A4253
:109CB00007D2DCE7094A9278022A04D1B3F5007F83
:109CC000D5D1FFF79BB8402BFBD9D0E7034A927858
:109CD000022A0CBF4FF480624022E8E759B400200A
:109CE0002DE9F047DDE9085681460C4690469A4634
:109CF0000027B84501DC01200EE06378052B04D174
:109D0000E37803F0030353450AD04FF0E023D3F880
:109D1000F03DDA0702D40020BDE8F08700BEFAE784
:109D200021464846FFF79EFF38B94FF0E023D3F8AD
:109D3000F03DDB07EFD500BEEEE7A378DA0914BFEC
:109D400033702B70237801371C44D2E70B4B01F0A2
:109D50007F0203EB420303EBD1112031487910F06D
:109D6000010008D14B795B0706D44B7943F004031B
:109D70004B71012070470020704700BF59B400208C
:109D80000B4B01F07F0203EB420303EBD1112031B7
:109D90004B7913F0010209D14B79C3F380005B07C3
:109DA00005D54B7962F382034B71704700207047F1
:109DB00059B4002070B5164D01F07F0605EB46053D
:109DC00005EBD11420346579ED0709D54FF0E02378
:109DD000D3F8F03DDA0701D4002070BD00BEFBE7E8
:109DE000657945F001056571FFF78EF80028F4D11B
:109DF000637960F300036371637960F382036371D5
:109E00004FF0E023D3F8F03DDB07E5D500BEE4E7F3
:109E100059B4002010B50C46FFF7C4F8094B04F004
:109E20007F0103EB410303EBD41191F8253043F09C
:109E3000020381F8253091F8253043F0010381F8C1
:109E4000253010BD59B4002010B50C46FFF7C0F8FE
:109E5000094B04F07F0103EB410303EBD41191F8AC
:109E600025306FF3410381F8253091F825306FF3E9
:109E7000000381F8253010BD59B40020054B01F0D6
:109E80007F0203EB420303EBD11191F82500C0F3ED
:109E90004000704759B400202DE9F04F87B001F021
:109EA00040F9002800F05E82DFF8CC92AD4B1D68CF
:109EB0002B78012B02D10020FEF786FF03A9281D75
:109EC000FFF704FD2B78012B044602D10020FEF79A
:109ED00075FF002C00F046829DF80D30013B072BEA
:109EE00000F27582DFE813F0080011006A024902EF
:109EF00054021B0015026C029DF80C00FFF76EFD6A
:109F0000994B9DF810209A70D0E79DF80C00FFF750
:109F100065FD964B002BC9D0FEF70CFCC6E7924CB2
:109F20009DF80C50237843F00103237094F82530FA
:109F30006FF3000384F8253094F825306FF3820323
:109F400084F8253094F826306FF3000384F8263027
:109F500094F826306FF3820384F82630002000F056
:109F6000CFFA9DF8106006F06002602A08D14FF029
:109F7000E023D3F8F03DD90740F1808100BE7DE1B8
:109F8000402A0DD17A48002800F0788100F0B8FA14
:109F900004AA00212846AFF30080002886D16DE195
:109FA00006F01F06012E00F04B81022E00F0718199
:109FB000002EDCD1202A11D19DF814300F2B00F295
:109FC0005D812344D878FFF7E9FC0146002800F0C2
:109FD000558104AA2846FFF72BFDDEE7002AC6D1EB
:109FE0009DF81130092BC2D801A252F823F000BF0E
:109FF0002BA20F001BA20F006F9F0F0009A20F00E2
:10A000006F9F0F0019A00F0093A10F006F9F0F000B
:10A0100033A00F0049A00F0004A800F077FA9DF8C4
:10A0200012102846FEF7D8FE237843F0020323706F
:10A030003CE763788DF80A3001230DF10A0204A988
:10A04000284600F021FA31E763789DF812A06BBB37
:10A05000BAF1000F2AD00AF1FF30C0B2FEF77AFA47
:10A0600010B14378022B08D04FF0E023D3F8F03D35
:10A07000DC077FF57CAF00BE79E7C379C3F38012BC
:10A08000C3F340131B0143EA4213227822F030024B
:10A09000134323704388C31800F109010093009B08
:10A0A0008B420AD8334B0BB1FEF741FB84F801A079
:10A0B00004A9284600F0D6F9F8E64B780B2B03BF2D
:10A0C0000B780F46C91800274B78042BCCD1009B86
:10A0D000A3EB01081FFA88F84FF0000B99F8003045
:10A0E0005FFA8BF60133B342BEDB3046FFF756FC16
:10A0F000424683680191284698470BF1010B01996C
:10A100000028EBD00828AFD98045ADD38B78234405
:10A11000DA78FF2AA8D1DE70D7B90A46002357782B
:10A12000052F08D192F802C00CF07F0704EB470717
:10A1300007EBDC17FE7417783B449BB298423A4415
:10A14000EDD899F8003001339E420144A7DD8BE73A
:10A15000BA788B789A4287D13A794B799A4283D1EF
:10A16000012312E094B4002059B4002035870F0079
:10A17000000000002F870F0058B4002091F802C0A3
:10A18000E21862440133D670DBB2FA789A42F5D80D
:10A19000C3E7BDF812309DF812001B0A013B0E2BDD
:10A1A0006CD8DFE803F008191F6B6B286B6B6B6BC7
:10A1B0006B6B6B6B1100FEF7C9F91223024604A901
:10A1C000284600F061F9E8E6854B002B56D0AFF346
:10A1D000008002465388F2E7FEF7BCF902460028E9
:10A1E000F8D1C4E6BDF81410FEF710FA02460028B4
:10A1F00044D01378E3E77B4B002B3FD0AFF30080D4
:10A2000002460028F5D1B2E6BDF81230012B35D157
:10A21000237843F0080323704AE7BDF81230012B7E
:10A220002CD123786FF3C303F5E72378C3F34012EF
:10A230009B0803F002031343ADF80A300223FCE647
:10A240009DF814300F2B19D82344D878FFF7A6FBBC
:10A25000014698B104AA2846FFF7EAFB00287FF4DC
:10A2600025AE9DF8103013F0600307D19DF8112042
:10A270000A2A3FF4DFAE0B2A3FF41AAF9DF80C0018
:10A280000021FEF78FFE9DF80C008021FEF78AFE6C
:10A290000CE69DF8141001F07F03082B3FF667AE23
:10A2A00004EB430303EBD113D87CFFF777FB07469E
:10A2B00022B10028E2D004AA01468BE69DF81130B5
:10A2C00003F0FD02012A08D0002B7FF450AE28468F
:10A2D000FFF7D4FDADF80A00B0E7BDF8122022B9AF
:10A2E000012B284612D1FFF7AFFD002F3FF4DEAD62
:10A2F00004AA39462846FFF79BFB002000F000F92E
:10A3000094F82630D8073FF5D1ADD1E6FFF782FDAE
:10A31000EBE79DF81010344B01F07F0403EB44038E
:10A3200003EBD11393F825006FF3000083F82500A9
:10A3300093F825006FF3820083F825003CB9059B54
:10A340009DF811209DF80C0000F0EEF8AEE5D87CE9
:10A35000FFF724FB48B94FF0E023D3F8F03DDA07CC
:10A3600000D500BE07B0BDE8F08F0469059B9DF8DD
:10A3700011209DF80C00A04798E51C4B002B3FF4E2
:10A3800095AD194B1878C0F3C000AFF300808DE590
:10A39000174B002B3FF48AADAFF3008086E5FFF743
:10A3A000FDFA436913B19DF80C009847013499F800
:10A3B0000030E0B201338342F1DA77E50024F6E7BA
:10A3C000049B002B3FF472AD059898476EE54FF063
:10A3D000E023D3F8F03DDB077FF568AD00BE65E50F
:10A3E000000000000000000059B400200000000040
:10A3F0000000000037B514490446CA89888991F9DC
:10A400000050831A9BB2402B28BF4023002D10DA46
:10A41000904214D01A4689680C48019300F0B2FEAD
:10A420000A4A019B8021204603B0BDE83040FFF777
:10A43000C1BC90424FF0000103D10022F3E780211C
:10A44000FBE7024AEFE700BF58B500206CB50020DB
:10A4500011F0800F4FF000031A460CBF80211946FF
:10A46000FFF7A8BC30B4074C05460B46086849689E
:10A47000224603C20022C4E902222846197830BCD1
:10A48000FFF7E6BF58B50020F8B5184E0C46054654
:10A4900008684968B260374603C70021F181E18846
:10A4A0008B4228BF0B46B381E18889B153B14AB9C9
:10A4B0004FF0E023D3F8F03DDA0701D40020F8BDD7
:10A4C00000BEFBE72846FFF795FF30B10120F6E715
:10A4D00021782846FFF7BCFFF7E74FF0E023D3F8D9
:10A4E000F03DDB07EAD500BEE9E700BF58B5002024
:10A4F000024814220021F9F715BF00BF58B500200B
:10A50000014B1861704700BF58B5002010B50246D6
:10A51000044C00685168234603C30023C4E9023396
:10A5200010BD00BF58B5002070B52D4C1E462378D5
:10A53000C909B1EBD31F054618D04EB14FF0E02347
:10A54000D3F8F03DDA0701D4002070BD00BEFBE770
:10A55000244B13B12146AFF3008023690BB90120CE
:10A56000F3E71F4A022128469847F8E794F900309C
:10A57000002B06DBA0680028E6D01B49324600F01D
:10A5800001FEA268E38932443344A260E2889BB2B0
:10A590009A42E38101D03F2E1ED823696BB92178FE
:10A5A0002846FFF755FF0028D9D14FF0E023D3F814
:10A5B000F03DDB07C8D500BEC7E70121084A2846A1
:10A5C000984701460028EAD12846FEF7EBFC802197
:10A5D0002846FEF7E7FCC2E72846FFF70BFFE2E755
:10A5E00058B50020000000006CB5002070B500F1E7
:10A5F000100504462846FFF757F93F2817D9E17898
:10A600000020FFF7A3FB90B12846FFF74DF93F2844
:10A61000E17807D904F638024023BDE870400020F5
:10A62000FFF7C8BBBDE870400020FFF7A9BB70BDB5
:10A6300008B5044B40F6B80202FB00301030FFF7BB
:10A6400019F908BDACB5002070B540F6B804074E46
:10A65000444304F1100092B23044FFF749F9054633
:10A660003019FFF7C3FF284670BD00BFACB500200E
:10A670002DE9F0410446FFF70BFA10B90020BDE8C0
:10A68000F081FFF70DFA06460028F7D140F6B80131
:10A69000164D4C4304F12408A8444046FFF7EAF85D
:10A6A0000028EBD02F193046B978FFF74FFB002870
:10A6B000E4D004F678042544294640224046FFF7BA
:10A6C00017F9B978044668B103462A463046FFF7C1
:10A6D00071FB48B94FF0E023D3F8F03DDB07CDD54F
:10A6E00000BECCE7FFF74CFB2046C8E7ACB5002026
:10A6F00070B50B4C40F6B80303FB0044243492B20F
:10A7000005462046FFF734F906462046FFF7B2F823
:10A710003F2802D92846FFF7ABFF304670BD00BF87
:10A72000ACB5002037B5144C40F6B80200212046E5
:10A73000F9F7F8FDFF234FF4424201256371E280EF
:10A740000023082263812273009304F138012B4611
:10A750004FF4806204F110002581FFF775F8009531
:10A760002B464FF4806204F5876104F12400FFF763
:10A770006BF803B030BD00BFACB5002010B50A4C7B
:10A78000002105222046F9F7CDFD04F11000243404
:10A79000FFF7F4F82046FFF7F1F820460121BDE865
:10A7A0001040FFF7F7B800BFACB50020F7B54B7904
:10A7B000022B064603D00025284603B0F0BD8B7956
:10A7C000022BF8D1204FBB787BBB8B783B700C7889
:10A7D00009250C4403E023781D44ADB21C44637882
:10A7E000242B1BD19542F6D96378042B12D16379BF
:10A7F0000A2B0FD1154B27780193013300930223C5
:10A800001A46E1193046FFF76BFA70B10E3517FAA8
:10A8100085F5ADB20C48FFF7E9FECDE7052BE3D196
:10A8200021463046FFF71EFA38B94FF0E023D3F83F
:10A83000F03DDB07BFD500BEBDE7A3787B70237872
:10A840001D44ADB21C44CFE7ACB50020AEB500202E
:10A8500070B50B461146127802F06002202A45D1ED
:10A86000234E8A883478944240D14A78203A032A89
:10A870003CD8DFE802F00213162F2BB91D4A07233C
:10A88000FFF702FE012070BD022BFBD11A4B002BFB
:10A89000F8D018490020AFF30080F3E7002BF1D186
:10A8A000ECE713B9FFF7DEFDECE7022BEAD14C88A9
:10A8B0001248347104F0010585F00101FFF76AF8D0
:10A8C0000F4B002BDED0C4F3400229460020AFF32B
:10A8D0000080D7E7002BE5D0022BD3D1094B002B0A
:10A8E000D0D049880020AFF30080CBE70020CAE732
:10A8F000ACB50020B2B5002000000000D0B50020AB
:10A9000000000000000000002DE9F347374D1C4611
:10A91000EB788B4207460E4607D0AB788B4258D176
:10A92000AB78B34232D001245CE0A2B205F6380124
:10A9300005F11000FFF71CF82D4B2BB92D4BEBB98F
:10A940002A48FFF753FEEBE76B79FF2BF6D005F6AD
:10A9500038094FF0000805F1100AA045EED019F8AB
:10A96000013B6A799A4206D15046FEF795FF10B92D
:10A970006979AFF3008008F10108EEE71E48FEF7A1
:10A980008BFF0028DCD1FDF747FAD9E71B4B13B149
:10A990000020AFF300800020FFF76AFE0028C2D13C
:10A9A0001748FEF767FF0028BDD1002CBBD014F07C
:10A9B0003F03B8D1A97801933846FFF7C7F9019B47
:10A9C00004460028AFD0A9781A463846FFF7F2F9B6
:10A9D00008E04FF0E023D3F8F04D14F0010401D06B
:10A9E00000BE0024204602B0BDE8F087ACB50020D0
:10A9F00000000000197E0F00BCB500200000000020
:10AA0000D0B5002073B5284CE28A52BA92B20546FE
:10AA10003AB94FF0E023D3F8F03DDB0739D500BE5B
:10AA200037E0A368B3FBF2F291B20029F1D0A06B3A
:10AA3000D4F811101B1AB3F5805F28BF4FF4805370
:10AA400092B209BAB0FBF2F6009302FB1602174B62
:10AA5000607B3144FDF7E4FC031E94F82E1012DAFB
:10AA6000A368A26B9B1AA362012384F82C3042F2E4
:10AA70000503A3872846002384F83E3002B0BDE8D2
:10AA80007040FFF7C7B906D100931A462846FFF772
:10AA9000C6F802B070BD054A9BB22846FFF78AF996
:10AAA0000028F6D1B5E700BF64CE002064BE0020C8
:10AAB00038B5184B184C0546A3B1607BAFF3008046
:10AAC00080B9A368A362012384F82C3042F2077393
:10AAD00084F83E0094F82F10A3872846BDE838403C
:10AAE000FFF798B9A26BA36894F82F109B1AB3F5DF
:10AAF000805F28BF4FF48053084A9BB22846FFF777
:10AB000059F930B94FF0E023D3F8F03DDB0700D519
:10AB100000BE38BD0000000064CE002064BE0020EE
:10AB2000044880F83C1080F83D2080F83E30012039
:10AB3000704700BF64CE0020024840220021F9F790
:10AB4000F1BB00BF64CE0020024840220021F9F78B
:10AB5000E9BB00BF64CE002073B54B79082B0546D6
:10AB600002D0002002B070BD8B79062BF9D1CB79D1
:10AB7000502BF6D1162A07D84FF0E023D3F8F03D3A
:10AB8000D907EED500BEECE7144C8B7884F82D3055
:10AB900004F12E030E78019304F12F030093022396
:10ABA0001A463144FFF79CF838B94FF0E023D3F848
:10ABB000F03DDA07D5D500BED4E794F82F101F2357
:10ABC00022462846FFF7F6F830B94FF0E023D3F8D5
:10ABD000F03DDB0700D500BE1720C3E764CE0020A0
:10ABE00037B50B460546144661B9127802F060028B
:10ABF000202A08D16278FE2A08D0FF2A03D12146F4
:10AC0000FFF730FC0123184603B030BD01238DF857
:10AC100007300A4B1BB1AFF300808DF807009DF899
:10AC20000730002BEFD0013B8DF807300DF1070204
:10AC3000012321462846FFF727FCE3E70000000038
:10AC40002DE9F041B04C94F83080B8F1010F90B08C
:10AC500005461E4600F0A081B8F1030F00F0078200
:10AC6000B8F1000F28D194F82F308B4201D0012089
:10AC70000EE02AB91F2E03D12068A44B98420AD0B7
:10AC80004FF0E023D3F8F03DD90700D500BE0020F7
:10AC900010B0BDE8F0819E4B23626368C4E90932BD
:10ACA000012384F83030A368C4E90D32E27B282AFE
:10ACB00012D12846FFF7A6FE94F83030022BD6D1E9
:10ACC00094F82E102846FFF7D9F8002800F0F881F4
:10ACD000002300931A46C4E12A2A03D12846FFF72D
:10ACE000E7FEE9E78BB1207BC0090ED1894A9BB210
:10ACF0002846FFF75FF80028DED14FF0E023D3F8B5
:10AD0000F03DDB07C3D500BEC2E7252A667B09D824
:10AD1000192A22D8032A00F00381122A00F0AB80FE
:10AD2000002A39D094F83C30002B00F01F8100231A
:10AD30006363012384F82C30022384F8303094F8C4
:10AD40003C30002B00F01C81A368002BB4D094F899
:10AD50002E102846FFF75EF8AEE71A3A00230B2ABA
:10AD6000E0D801A151F822F0C9AE0F00BBAD0F0031
:10AD700025AD0F0025AD0F0025AD0F0025AD0F004F
:10AD800025AD0F0025AD0F0025AD0F0033AE0F0030
:10AD900025AD0F00D7AD0F003046FDF72DFB002885
:10ADA00040F0F48094F83C30002BBBD140F20243D9
:10ADB000A387002384F83E30B4E7574B002B00F004
:10ADC000E580E17C3046C1F3400301F0010209094E
:10ADD000FDF7BAFBE3E70DF1160206A93046FDF7D1
:10ADE000ABFB069B13B1BDF816203AB994F83C3082
:10ADF000002B97D140F20242A287DBE712BA013B57
:10AE00001BBA089243480793082207A900F0BAF931
:10AE100008200022606384F82C20002800F0B8800D
:10AE2000A36898423FF62CAF3A4A94F82E1083B2AA
:10AE30005EE7CDE90733099308238DF81F300DF144
:10AE40001602022306A930468DF82430FDF774FB64
:10AE5000069A002ACAD0BDF81630002BC6D012BA06
:10AE600008925BBA2B48ADF826300C2207A900F0F7
:10AE700089F90C20CDE72422002107A8F9F752FA1E
:10AE800080238DF81D3008220223202109A88DF887
:10AE90001E308DF81F30F9F745FA102220210BA83B
:10AEA000F9F740FA042220210FA8F9F73BFA0FAB7B
:10AEB0000BAA09A93046FDF76BFA1648242207A908
:10AEC00000F060F92420A4E78DF81D308DF81E30C5
:10AED0008DF81F30114B03228DF81C208BB13046AA
:10AEE000AFF300809DF81E3080F0010060F3C713BF
:10AEF000042208488DF81E3007A900F043F9042009
:10AF000087E70120EEE700BF64CE0020555342439F
:10AF10005553425364BE002049850F0000000000D5
:10AF20001222002107A8F9F7FDF9F02394F83C203C
:10AF30008DF81C300A238DF823304FF0000362F3A4
:10AF400003038DF81E3094F83D308DF828306748A3
:10AF500094F83E308DF82930122207A900F012F93A
:10AF60000023A38784F83E30122052E7A38E5F4A65
:10AF70005F49607BFDF742FA0028FFF6D8AE48E74C
:10AF800042F20502A28784F83E30DDE6002040E769
:10AF9000022384F830308FE6277BFF0915D1E37B4D
:10AFA000607B2A2B27D0A38E504A04F10F01FDF7B6
:10AFB00025FA0028BFBF42F2050384F82C80A3873E
:10AFC00084F83E70A8BF84F82C70A36B1E44636B9A
:10AFD000A6639E42DCD2E37B282B3FF46AAE2A2B89
:10AFE0003FF47CAE4FF0E023D3F8F03DDA077FF575
:10AFF00063AE00BE60E6E38AD4F81110D4F838C01E
:10B0000000965BBA9AB209BAA368B3FBF2F39AB29C
:10B01000364BBCFBF2FE02FB1EC27144FDF722FA66
:10B020000028324B0EDAA368A26B84F82C809B1A9E
:10B03000A362022384F8303042F20503A38784F828
:10B040003E7039E68642C0DD321A40B1A16B0392F0
:10B050000144A1631918184600F0A2F8039A0023CE
:10B06000009394F82F102846FEF7D9FDFFE594F8D9
:10B070002E308B427FF420AE0D2E7FF41DAEE37B8D
:10B08000282B09D02A2B14D01A4B53B1607B04F122
:10B090000F01AFF3008004E0174B13B1607BAFF3F7
:10B0A0000080002384F83030144A94F82F101F23B6
:10B0B0001EE6134B002BF4D0607BFDF7EBF9F0E7B5
:10B0C00094F82F102846FEF7D9FE00287FF400AE32
:10B0D000032384F830300B4A94F82E100D232846B1
:10B0E000FEF768FE00287FF4C2AD06E664BE0020CD
:10B0F00073CE0020000000000000000064CE00209D
:10B1000095840F0084CE002008B50020FEF7D6FC01
:10B1100030B94FF0E023D3F8F03DDB0700D500BE97
:10B1200008BDFEF7C5BC00000649074A074B9B1A3D
:10B1300003DD043BC858D050FBDCF9F7F1FFF9F709
:10B1400083F80000DCB70F0000800020C4860020D8
:10B15000FEE7FEE7FEE7FEE7FEE7FEE7FEE7FEE7C7
:10B16000FEE7FEE710B501390244904201D100200C
:10B1700005E0037811F8014FA34201D0181B10BD60
:10B180000130F2E70A44914200F1FF3300D17047E9
:10B1900010B511F8014B03F8014F9142F9D110BDE0
:10B1A000884210B501EB020402D98442234607D835
:10B1B000431EA14208D011F8012B03F8012FF8E734
:10B1C000024401468A4200D110BD13F8014D02F835
:10B1D000014DF7E710B50246147813460132002CF2
:10B1E000FAD1013B11F8012B03F8012F002AF9D104
:10B1F00010BD034613F8012B002AFBD1181A0138A1
:10B2000070470000F0B51F4C8BB005460B466E46EC
:10B2100004F1200C20686168374603C70834644590
:10B220003E46F7D121793971911E20683860222974
:10B230004FF0000104D919700B4618460BB0F0BD51
:10B24000581E8446B5FBF2F702FB175628366E44AB
:10B250000C4616F8286C0CF8016F2E46B24201F12C
:10B2600001013D46EED900225A541919A51AAA42E5
:10B27000E3DA10F8015F0E780670013201F8015927
:10B28000F4E700BFA8B70F00FFF7BCBF53B94AB936
:10B29000002908BF00281CBF4FF0FF314FF0FF30DE
:10B2A00000F074B9ADF1080C6DE904CE00F006F8B9
:10B2B000DDF804E0DDE9022304B070472DE9F04732
:10B2C000089D04468E46002B4DD18A42944669D98A
:10B2D000B2FA82F252B101FA02F3C2F1200120FA6D
:10B2E00001F10CFA02FC41EA030E94404FEA1C48BB
:10B2F000210CBEFBF8F61FFA8CF708FB16E341EAB7
:10B30000034306FB07F199420AD91CEB030306F13C
:10B31000FF3080F01F81994240F21C81023E63445D
:10B320005B1AA4B2B3FBF8F008FB103344EA034401
:10B3300000FB07F7A7420AD91CEB040400F1FF3316
:10B3400080F00A81A74240F207816444023840EA53
:10B350000640E41B00261DB1D4400023C5E900438C
:10B360003146BDE8F0878B4209D9002D00F0EF800F
:10B370000026C5E9000130463146BDE8F087B3FA42
:10B3800083F6002E4AD18B4202D3824200F2F9802A
:10B39000841A61EB030301209E46002DE0D0C5E92D
:10B3A000004EDDE702B9FFDEB2FA82F2002A40F079
:10B3B0009280A1EB0C014FEA1C471FFA8CFE01267C
:10B3C000200CB1FBF7F307FB131140EA01410EFB20
:10B3D00003F0884208D91CEB010103F1FF3802D2C7
:10B3E000884200F2CB804346091AA4B2B1FBF7F0C1
:10B3F00007FB101144EA01440EFB00FEA64508D9E4
:10B400001CEB040400F1FF3102D2A64500F2BB8020
:10B410000846A4EB0E0440EA03409CE7C6F120076F
:10B42000B34022FA07FC4CEA030C20FA07F401FAB5
:10B4300006F31C43F9404FEA1C4900FA06F3B1FB3E
:10B44000F9F8200C1FFA8CFE09FB181140EA0141A3
:10B4500008FB0EF0884202FA06F20BD91CEB010140
:10B4600008F1FF3A80F08880884240F28580A8F198
:10B4700002086144091AA4B2B1FBF9F009FB1011EA
:10B4800044EA014100FB0EFE8E4508D91CEB010188
:10B4900000F1FF346CD28E456AD90238614440EA2B
:10B4A0000840A0FB0294A1EB0E01A142C846A646AB
:10B4B00056D353D05DB1B3EB080261EB0E0101FA34
:10B4C00007F722FA06F3F1401F43C5E90071002691
:10B4D0003146BDE8F087C2F12003D8400CFA02FCE7
:10B4E00021FA03F3914001434FEA1C471FFA8CFEF7
:10B4F000B3FBF7F007FB10360B0C43EA064300FBE7
:10B500000EF69E4204FA02F408D91CEB030300F184
:10B51000FF382FD29E422DD9023863449B1B89B23B
:10B52000B3FBF7F607FB163341EA034106FB0EF3C4
:10B530008B4208D91CEB010106F1FF3816D28B4271
:10B5400014D9023E6144C91A46EA004638E72E463D
:10B55000284605E70646E3E61846F8E64B45A9D235
:10B56000B9EB020864EB0C0E0138A3E74646EAE7A4
:10B57000204694E74046D1E7D0467BE7023B614452
:10B5800032E7304609E76444023842E7704700BFBB
:10B59000F8B500BFF8BC08BC9E467047F8B500BFC0
:10B5A000F8BC08BC9E4670470080002000100200D6
:10B5B0000338FDD8704700000000000000000000C4
:10B5C0000338FDD8704701000000000008990020F2
:10B5D0000338FDD870474164614446550052414BE1
:10B5E000576972656C65737300576973426C6F635A
:10B5F0006B2052414B3436333100302E342E320919
:10B60000207331343020362E312E310000000000FE
:10B6100000000000000000000000000023D1BCEA90
:10B620005F782315DEEF12120000000070B00020DA
:10B630004164616672756974006E524620554632E7
:10B64000003031323334353637383941424344459E
:10B6500046006E52462053657269616C00090453BE
:10B660006F66744465766963653A200053002E0066
:10B670006E6F7420666F756E640D0A00EB3C90551A
:10B6800046322055463220000201010002400000EF
:10B6900000F80201010001000000000009010100A2
:10B6A0008000294200420052414B343633310000C1
:10B6B000000046415431362020203C21646F6374E1
:10B6C0007970652068746D6C3E0A3C68746D6C3EE0
:10B6D0003C626F64793E3C7363726970743E0A6CBD
:10B6E0006F636174696F6E2E7265706C616365283B
:10B6F0002268747470733A2F2F73746F72652E7290
:10B70000616B776972656C6573732E636F6D2F6300
:10B710006F6C6C656374696F6E732F776973626C9D
:10B720006F636B2D636F726522293B0A3C2F736335
:10B73000726970743E3C2F626F64793E3C2F68746E
:10B740006D6C3E0A00000000494E464F5F55463280
:10B750005458540020850020494E4445582020204C
:10B7600048544D00BAB60F0043555252454E54202E
:10B77000554632000000000025A70F007DA70F00EE
:10B78000ADA70F0051A80F0009A90F00000000008D
:10B7900039AB0F0049AB0F0059AB0F00E1AB0F0005
:10B7A00041AC0F0000000000303132333435363701
:10B7B00038396162636465666768696A6B6C6D6E6F
:10B7C0006F707172737475767778797A0000000003
:04B7D0000000000075
:08B7D4006C8AFF7F01000000F8
:10B7DC0000000000EC82002054830020BC83002079
:10B7EC00000000000000000000000000000000004D
:10B7FC00000000000000000000000000000000003D
:10B80C00000000000000000000000000000000002C
:10B81C00000000000000000000000000000000001C
:10B82C00000000000000000000000000000000000C
:10B83C0000000000000000000000000000000000FC
:10B84C0000000000000000000000000000000000EC
:10B85C0000000000000000000000000000000000DC
:10B86C0000000000000000000000000000000000CC
:10B87C0000000000000000000100000000000000BB
:10B88C000E33CDAB34126DE6ECDE05000B00000080
:10B89C00000000000000000000000000000000009C
:10B8AC00000000000000000000000000000000008C
:10B8BC00000000000000000000000000000000007C
:10B8CC00000000000000000000000000000000006C
:10BBFC000000000000000000E0860020FFFFFFFFB7
:10BC0C007C7F00200090D003FF00FFFF320000007B
:10BC1C00FD7C0F00717D0F00010902620003010021
:10BC2C008032080B0002020200000904000001022D
:10BC3C000200040524002001052401000104240253
:10BC4C000205240600010705810308001009040100
:10BC5C0000020A00000007050202400000070582EE
:10BC6C000240000009040200020806500507050303
:10BC7C00024000000705830240000009024B00024D
:10BC8C0001008032080B00020202000009040000CF
:10BC9C000102020004052400200105240100010416
:10BCAC00240202052406000107058103080010097F
:10BCBC00040100020A000000070502024000000710
:10BCCC0005820240000012010002EF0201409A239B
:10BCDC0029000001010203015DB60F00DDB50F0064
:10BCEC00E9B50F0064B3002052B60F0039B60F004F
:10BCFC0055463220426F6F746C6F616465722030F0
:10BD0C002E342E3209206C69622F6E7266782028D0
:10BD1C0076322E302E3029206C69622F74696E7940
:10BD2C007573622028302E31302E312D3239332D5F
:10BD3C0067616638653561393029206C69622F7509
:10BD4C006632202872656D6F7465732F6F72696728
:10BD5C00696E2F636F6E6669677570646174652DAB
:10BD6C00392D6761646262386337290D0A4D6F643F
:10BD7C00656C3A20576973426C6F636B2052414B70
:10BD8C003436333120426F6172640D0A426F617236
:10BD9C00642D49443A20576973426C6F636B2D5282
:10BDAC00414B343633312D426F6172640D0A44615C
:10BDBC0074653A204E6F7620333020323032310D9C
:10BDCC000A0000000000000000000000000000005D
:10BDDC000000000000000000000000000000000057
:10BDEC000000000000000000000000000000000047
:10BDFC000000000000000000000000000000000037
:10BE0C000000000000000000000000000000000026
:10BE1C000000000000000000000000000000000016
:10BE2C000000000000000000000000000000000006
:10BE3C0000000000000000000000000000000000F6
:10BE4C0000000000000000000000000000000000E6
:10BE5C0000000000000000000000000000000000D6
:10BE6C0000000000000000000000000000000000C6
:10BE7C000100000098B4002010000C000000E0FF4E
:10BE8C001F00000000000000C9430F0025420F00F6
:04BE9C0001420F0050
:10D80000F1109E1E797A22200500000064000000BD
:10D81000CC00000000001000CD000000000004005B
:10D82000D000000029009A23D10000004028A5ADB7
:10D83000D2000000200000000000000000000000F6
:10D8400000000000000000000000000000000000D8
:08D850000000000000000000D0
:020000020000FC
:020000041000EA
:0410140000400F0089
:0410180000E00F00E5
:04000003F000B1292F
:00000001FF
